:1000000002755902782300000000000271CF000041
:1000100000000002788100000000003200000000B3
:10002000000000023E4800000000000272F90000DB
:1000300000000000000000000000000000000000C0
:100040005052343032207665722E3132382E312EB5
:1000500030204864773A482032302D30362D303504
:100060002032333A3232202075F00612011E22125D
:100070006E9375F00612011E126E982212006F1216
:10008000006812006F12006812006F120068120000
:100090006F12006812006F75F01812011E22126EA6
:1000A0009375F04B12011E126E982275510412388E
:1000B00012123828126E9375F0C812011E126E9833
:1000C0002275510512381212382812009E75F01E42
:1000D00012011E12009E2275510712381212382882
:1000E0001200882275510612381212382812008E1A
:1000F0002212007C12007C221200E41200E41200A2
:10010000E422C2A1C25812006F75F01212011ED271
:10011000A1C2582212006F75F01212011E22128223
:10012000E9201607C0F0123268D0F0D5F0F0227046
:1001300004A243B322C0E01412013ED0E022C0E08A
:10014000030303540F28F8D0E0C0E0540704F5F08F
:10015000E213D5F0FCD0E0227003D3802830E7030F
:10016000C3802223F9C3137004A243801814C0E093
:10017000030303540F2479F8D0E0540704F5F0E2A8
:1001800013D5F0FCE992E022C0E024B4F8E21201B9
:10019000584004D0E0C322D0E024CAF58274003471
:1001A00000F583E01201A82220E702C322C2E7C0C3
:1001B000E0C2E0700AA243B3D0E030E001B322B461
:1001C0007E03C380F3B40204A22380ECB40404A22F
:1001D0002480E5B40604A22580DEB40804A22B80A6
:1001E000D7B40A04A20A80D0B40C0AE5774578C3D4
:1001F0006001D380C3B40E0512715180BBB41007E7
:10020000A25E725DB380B1B41206A25D822680A8A0
:10021000B41406A25DB026809FB41604A25E809836
:10022000B418077400127E56808EB41A0774011237
:100230007E568084B41C087402127E560201B8B443
:100240001E087403127E560201B8B420087404120A
:100250007E560201B8B422087405127E560201B817
:10026000B424087406127E560201B8B42608740736
:10027000127E560201B8D0E0C3221243F4E56E604C
:1002800013B4010512333E8008B4020512335180C5
:1002900000756E00123268E5795440600B20A808A2
:1002A000305505C255123382127CAB22C2B612778A
:1002B000CC75380074031258EEE51E1258EEE51F97
:1002C0001258EE74571258EE1202D5E5381258EE55
:1002D0003099FDD3227885E6232354031258EE7813
:1002E00086E630E402240A540F1258EE7885E6C4FC
:1002F000540375F00AA4F5F0E6540F25F01258EEF9
:100300007884E6C4540375F00AA4F5F0E6540F258A
:10031000F01258EE7883E6C4540775F00AA4F5F09D
:10032000E6540F25F01258EE7882E6C4540775F0B3
:100330000AA4F5F0E6540F25F01258EE7886E6038D
:10034000C454071258EE22C0F075F0DCD5F005B2A7
:10035000B5126ACAC0F0120591D0F030E7EED0F0C5
:1003600022AAF0120347E5336530F5F0E534653134
:1003700045F0600C1204B8853033853134120347E0
:1003800012055612034712057E1203471204C58A4E
:10039000F022AAF0120347E5336530F5F0E5346545
:1003A0003145F0600C1204B88530338531341203C6
:1003B0004712054212034712057E1203471204C575
:1003C0008AF02279207530017531037532E0900092
:1003D000E01203471204B81203471205167900759C
:1003E0003001753104753200900100120347120488
:1003F000B812034712051679E0753001753105759D
:1004000032009002001203471204B812034712058B
:100410001685303385313422AAF0120347E533655F
:1004200030F5F0E534653145F0600C1204B88530E4
:10043000338531341203471204FE8AF022AAF012E7
:100440000347E5336530F5F0E534653145F0600C80
:100450001204B88530338531341203471204E68A1A
:10046000F022C0F075F00833C297928300D297D57E
:10047000F0F5D0F022C0F075F008C297D29700A234
:100480008233D5F0F5D0F022D2B7D297D283D28280
:10049000D28422E53133E5303322C3E5313322E51E
:1004A000322212046212049312046212049A120499
:1004B0006212049F12046222120488C284745312CE
:1004C00004A2D28422120488C28474581204A2D2D4
:1004D0008422120488C28474541204A2E4120462B6
:1004E000120475D28422120488C28474541204A2A5
:1004F000E4120462120475F608D9F9D284221204B7
:1005000088C28474541204A2E4120462120475F2C4
:1005100008D9F9D28422120488C28474541204A225
:10052000E4120462120475F0A3D9F9D284221204F1
:1005300088C0E0C28474841204A2D0E0120462D2A3
:100540008422120488C28474841204A2E612046213
:1005500008D9F9D28422120488C28474841204A2B5
:10056000E212046208D9F9D28422120488C2847487
:10057000841204A2E0120462A3D9F9D284221204E4
:1005800088C28474831204A2D2841282E91282E99E
:1005900022C2847457120462120475D28422D28358
:1005A000D282D297D2B7D284B2B575F0021282E964
:1005B000D5F0FAC2B7B2B575F0021282E9D5F0FAF9
:1005C000D2B7B2B5227530017531DB753200120336
:1005D000471208607533FF7534FF22AE83AD8290F9
:1005E000DB007F207404F97480F875300185833155
:1005F00085823212043D7880E66E702508E66D70C3
:100600002008E6601AB4FF028013167404F974809F
:10061000F8753001858331858232120392C322D36B
:1006200022A3A3A3A3DFBD80F490DB007F2074048A
:10063000F97480F875300185833185823212043D6A
:100640007880E66E700908E66D700408E6FC22A367
:10065000A3A3A3DF0A7CFF2290DB007F207BFF7433
:1006600004F97480F8753001858331858232120473
:100670003D7880E66E702C08E66D702708ECB4FFBC
:100680000D788076FF0876FF0876FF0874FFF67411
:1006900004F97480F8753001858331858232120344
:1006A00092C322BBFF107880E6B4FF0A08E6B4FFCD
:1006B00005C374209FFBA3A3A3A3DFA3BBFF02D3A7
:1006C00022EB232354FC2400F5827583DB500205C2
:1006D000837880EEF608EDF608ECF608E4F674048C
:1006E000F97480F875300185833185823212039266
:1006F000C32275830075F08E7530028583317532A3
:1007000000C0F0C083120347120860D0830583D075
:10071000F0D5F0E475830075F0DA75300385833128
:10072000753200C0F0C083120347120860D0830501
:1007300083D0F0D5F0E47533FF7534FF2275830064
:1007400075820075F08EC0F0C082C083753002855E
:1007500083317532001203471204B8D083D082C0AF
:1007600082C08375300085823175320012034712D2
:10077000057ED083D08205830582D0F0D5F0C77581
:10078000830075820075F0DAC0F0C082C0837530D6
:10079000038583317532001203471204B8D083D029
:1007A00082C082C0837530018582317532001203A8
:1007B0004712057ED083D08205830582D0F0D5F024
:1007C000C77533FF7534FF2275830075820075F09D
:1007D0008EC0F0C082C083753000858331753200D1
:1007E0001203471204B8D083D082C082C083753010
:1007F0000285823175320012034712057ED083D004
:100800008205830582D0F0D5F0C77583007582001C
:1008100075F0DAC0F0C082C0837530018583317510
:1008200032001203471204B8D083D082C082C08342
:1008300075300385823175320012034712057ED070
:1008400083D08205830582D0F0D5F0C77533FF755C
:1008500034FF22120488C28474501204A2D284226B
:10086000120488C28474811204A2D28422120488E1
:10087000C28474841204A2E8120462D9FAD28422D7
:10088000F8790012034712086DEAC0E085823085CE
:10089000833175320012034712057ED0E0FA0583DA
:1008A000DAE77533FF7534FF22120488C28474546A
:1008B0001204A2E4120462E4C0E0120475D0F02530
:1008C000F0D9F5D284227583007582028006758383
:1008D00000758200E475F08D858230858331753234
:1008E00000C082C083C0F0C0E01203471204B812F7
:1008F000034779001208A9D0F025F0D0F0D083D0BA
:10090000820583D5F0D2858230858331753200C06F
:10091000E01203471204B812034779201208A9D045
:10092000F025F07533FF7534FF227583007582035F
:100930008006758300758201E475F0DA8582308562
:100940008331753200C082C083C0F0C0E01203471B
:100950001204B812034779001208A9D0F025F0D08C
:10096000F0D083D0820583D5F0D27533FF7534FF84
:1009700005E02275830075F00075300085833175C0
:100980003200C0F0C083120347120860D083058391
:10099000D0F0D5F0E47533FF7534FF75830075F042
:1009A000DA753001858331753200C0F0C0831203DF
:1009B00047120860D0830583D0F0D5F0E47533FF8B
:1009C0007534FF2253590F53580F5318F053190F12
:1009D000C2AFE5582324B1F8E5184519F608A61A60
:1009E000055853580FE558B55905055953590FD2B5
:1009F000AFC3E55895595002241024F45003756391
:100A00000022E559B558057400780022C33324B19B
:100A1000F8E6C0E008E6F8D0E02253580F53590F2B
:100A2000C2AFE559B55804D2AFD322055953590F77
:100A3000D2AFC380F53008597885E6540FC0E0E6A0
:100A4000C4540375F00AA4D0F025F0FD7886E63092
:100A5000E402240A540FFE901A007F3C7404F974D7
:100A600000F87530018583318582321204187800D0
:100A7000E26D701708E26E701208E2C42354E0F5CC
:100A8000F07886E6541F45F0F68006A3A3A3A3DF03
:100A9000CB221277CC120A351277DBFEAFF07DFF46
:100AA0000DED30E70122D26575F004A424E0F58253
:100AB000E5F03400F583C082C0837880E0F6A308B7
:100AC000E0F6A308E0F6A308E0F6D083D0827880B1
:100AD00086830886827880B6FF0708B6FF03020B7C
:100AE00058C3E58233F582E58333F583E58224E05C
:100AF000F582E5833405F5837882E6705B08E6606D
:100B000057FB7402F97480F8753001858331858252
:100B10003212043DA3A37880E60856B4FF03020B0B
:100B200058788086F053F07F08E6C39EC5F09F405A
:100B30001E7025E5F06018BD001E20431B7880E67E
:100B4000A2E720E713E5F024FA400DD2748009787B
:100B500080E6A2E79265DBAABD00028028ED14C002
:100B6000E0030303540F2479F8D0E0540704FB7426
:100B700000D333DBFD306505FBE24B8004F4FBE280
:100B80005BF2020AA0B2651232B5406F20316C20D0
:100B9000170B204205306563800320655E30653C9D
:100BA00020423978B3E2702E20732078B1E2602CB5
:100BB00012751A6027F5F07518C0751909E5F0541B
:100BC0003F4400F51A1209C4020BD012751A600CCA
:100BD00078B1E278B3F2D274D273801FC274C27358
:100BE000A2659242400D304312C24312336012524A
:100BF0008D8008204305D243123373020AA01204E9
:100C00006212049312046212049AD2E01204621275
:100C1000049F12046222120488C2847454120BFED0
:100C2000E4120462120475F608D9F9D2842212047F
:100C300088C2847484120BFEE612046208D9F9D2C9
:100C4000842290FC00753004753100753200C0823A
:100C5000C083754BFA1203471204B885306D853195
:100C60006C79087880120347120C16120E3ED0835E
:100C7000D0827044C082C0837884868308868212C2
:100C80000CEF402478828683088682120CEF40188D
:100C9000120D0EE582600AE56AB56C0CE56BB56D68
:100CA00007D083D082020CCA7882E6249AF6120E0C
:100CB00081126789D083D0820531E5317002053019
:100CC000A3E58245837087120CD17533FF7534FF1D
:100CD000227882760008760078847600087600080C
:100CE0007600087600756D04756C00120E5D22C0EA
:100CF00082C083E5822400F582E5833480F5834059
:100D000005D083D08222D083D08290000022E58259
:100D100075F008A4F582E5F0C58375F008A4258375
:100D2000F583E5F03404F56BE5822400F582E58374
:100D30003400F5835002056B85836A22126799D0CF
:100D400083D08222C082C083120E1770EF78828611
:100D500083088682120CEF40E3120D0E1210F87811
:100D60008076007884E518F608E519F6087600081C
:100D700076007408F97480F8856B3085833185823C
:100D8000321203927404F97484F8856B30858331D0
:100D900085823212043D75F00478807984E66760BC
:100DA0000280990809D5F0F5120E1E788286830814
:100DB0008682A3120CEF7882A68308A682788486A6
:100DC00083088682120CEF7882E66583700A08E653
:100DD00065827004A3120CEF7884A68308A682C0F3
:100DE0006DC06C856B6D856A6C120E5DD0E0D0F0C5
:100DF000B56C09C5F0B56D028018C5F0C06DC06C4A
:100E000085F06DF56C7882E62499F6120E81D06C2F
:100E1000D06DD083D08222120E1E120E3E22856D1E
:100E200030856C317532001203471204B8790878A6
:100E300080120347120C16853033853134227885B1
:100E4000E618261826182618245566700F7885E6A9
:100E500018661866186618661864996622120E6479
:100E6000120E81227885E618261826182618245591
:100E7000F67885E61866186618661866186499F696
:100E800022856D30856C317532001203471204B82B
:100E900012034779087880120C2E12034712057E40
:100EA0001203471204C585303385313422120E17E0
:100EB00070307882E6C0E008E6C0E00886830886E5
:100EC00082C3D0E09582F582D0E09583F5835010FF
:100ED0004582600CE5822400F582E5833480F58349
:100EE000C322900000D322C2B6120EADE433C0E09C
:100EF00075380074031258EEE51E1258EEE51F1205
:100F000058EE74531258EED0E01258EE7400125896
:100F1000EE74001258EEE5831258EEE5821258EE98
:100F2000E5381258EE3099FD22C2B6E5366004F479
:100F3000FF8004FF120CD175380074031258EEE5DF
:100F40001E1258EEE51F1258EE74561258EEEF12AC
:100F500058EEE5381258EE3099FD227401C0E07861
:100F60008075F008E4F608D5F0FBD0E0D322120E2D
:100F7000AD40E860E878848683088682120F81C3DA
:100F800022C082C083E58275F008A4F582E5F0C531
:100F90008375F008A42583F583E5F03404F56BE54B
:100FA000822400F582E5833400F5835002056B74DA
:100FB00008F97480F8856B3085833185823212049C
:100FC0003DD083D08222120EAD7F085005120CD185
:100FD0007F007882865A08865B08865C08865DC238
:100FE000B675380074031258EEE51E1258EEE51F70
:100FF0001258EE74541258EEE5361258EEEF1258AD
:10100000EEE536603CE55D655BF5F0E55C655A450F
:10101000F0600B855D82855C83120F818003120F67
:101020005D855D82855C83A3120CEF85825D85837F
:101030005C788075F008E61258EE08D5F0F8D536E1
:10104000C4E5381258EE3099FDC322E5367007C268
:10105000AF120EAD5005E536F4800C7884A65C081E
:10106000A65D120E5DE536D2AFC0E0C2B67538009F
:1010700074031258EEE51E1258EEE51F1258EE7476
:10108000551258EED0E01258EEE5381258EE30996D
:10109000FDD322C2B675380074031258EEE51E1255
:1010A00058EEE51F1258EE74581258EE74202323A0
:1010B00054FC041258EE74201258EE90DB007F208E
:1010C0007404F97480F87530018583318582321299
:1010D000043D7880E61258EE08E61258EE08E61253
:1010E00058EE08E61258EE08A3A3A3A3DFD2E53812
:1010F0001258EE3099FDD3221277CC7886E630E490
:1011000002240A540FC4F97885E6C4540375F00A22
:10111000A4F5F0E6540F25F0C313497881F67885DD
:10112000E692E754C0F97883E6C4540775F00AA440
:10113000F5F0E6540F25F049F97884E6C4540375B8
:10114000F00AA4F5F0E6540F25F0F5F07882E654A5
:10115000702345F07883F67882E9F622223044FD48
:10116000126E9375F00612011E126E9875F014122D
:10117000011EE540C24422C0E0858330858231757E
:1011800032001203471204B8753003D031753200B3
:1011900012034712057E7533FF7534FF22C082C0EB
:1011A00083753003F5317532001203471204B8D04D
:1011B00083D08285833085823175320012034712D5
:1011C000057E7533FF7534FF22745578807910F6EB
:1011D00008D9FC7410F97480F885833085823175E4
:1011E00032001203927533FF7534FF7410F9748066
:1011F000F885833085823175320012043D7880791C
:1012000010B6553B76AA08D9F87410F97480F885A1
:1012100083308582317532001203927533FF753445
:10122000FF7410F97480F88583308582317532003F
:1012300012043D78807910B6AA0508D9FAE4227420
:10124000012275F000C0F0900000C082C08374DB02
:10125000121177D083D082C082C0831211C9600777
:10126000D0F075F001C0F0D083D082C082C083740A
:10127000DB12119DD083D082A37400B583CC74405F
:10128000B582C7D0E02278807910E6B5F00708056E
:10129000F0D9F7E422740122C0E078807910F608D2
:1012A00005E0D9FA7410F97480F87530037531DBF4
:1012B0007532001203927410F97480F8753003755A
:1012C00031DC7532001203927410F97480F87530B5
:1012D000037531DB75320012043DD0F0C0F01212FC
:1012E00086701E7410F97480F87530037531DC75E2
:1012F000320012043DD0F0C0F01212867003D0F01C
:1013000022D0F022E51DC0E0121298D0F07006E560
:10131000F0F4121298227564FF121476C2081209B2
:10132000326001221203C37401F97464F87530014C
:101330007531037532A012043D7410F97489F87583
:1013400030017531037532C01204187410F97499A4
:10135000F87530017531037532D01204187402F932
:101360007466F87530017531CE7532001204187448
:1013700016F974B4F87530017531CE7532C01204A7
:101380001878B49000CA75F016E2F008A3D5F0F909
:101390007416F974B4F87530017531037532A11201
:1013A00004187408F97400F87530017531D275327B
:1013B0000012041878009002F375F008E2F008A318
:1013C000D5F0F9D208E422798077E909E4A22692DF
:1013D000E0A22792E1A22892E2A22C92E3A24292FA
:1013E000E4F709A73909A73A09A73B7404F97480FF
:1013F000F875300275318E75320012039222D24296
:10140000D243C221C227A227B392A5C222C228A2D8
:1014100028B392A6C22AC22CA22CB39280227404B2
:10142000F97480F875300275318E75320012043D02
:101430007880B6E9C908E6A2E092269220B392A786
:10144000A2E192279221B392A5A2E292289222B31E
:1014500092A6A2E3922A922CB39280A2E4924278BE
:101460008076FF7401F97480F875300275318E75DD
:1014700032001203922278B475F016E4F208D5F027
:10148000FB74FF78BCF278BDF222E8C0E07861E23C
:10149000F572D0E0F822E8C0E07862E2F572D0E0C0
:1014A000F822E8C0E07863E2F572D0E0F82275F047
:1014B0000384B40104741A8017B4020474228010E7
:1014C000B40304742A8009B4040474428002741AB8
:1014D000227403F9745EF875300075318C7532E54D
:1014E000120418785EE21214AE7861F2785FE212AC
:1014F00014AE7862F27860E21214AE7863F2785E2D
:10150000E224FD9201E224E292027401F9745DF892
:1015100075300075318C7532E2120418785DE22462
:10152000FD9204E224E29205227403F9745EF875D8
:10153000300075318C7532E51203617401F9745D08
:10154000F875300075318C7532E2120361227980B2
:10155000774809774E0977800977A07404F9748079
:10156000F875300075318D7532201203927404F9CC
:101570007480F875300275318D7532201203922215
:101580007404F97480F875300075318D753220124D
:10159000043D7982E7648022E4A21C92E0A21D92BD
:1015A000E1A21E92E2A22992E37980F77401F97414
:1015B00080F875300075318C7532E8120392227410
:1015C00001F97480F875300075318C7532E81204B9
:1015D0003D7980E7A2E0921CA2E1921DA2E2921E58
:1015E000A2E39229227980E4A22D92E0A22E92E138
:1015F000A22F92E2A21492E392E492E5A23192E643
:1016000092E7F709E4A23092E0A23292E1A233928B
:10161000E2A23492E3A23692E6A23792E7F709E417
:10162000A23892E0A23A92E2A23B92E3A23C92E478
:10163000A23D92E5A23E92E7F709E579F77404F935
:101640007480F875300075318C7532EC1203927924
:1016500080E57AF4F709E57BF4F709E57CF4F774A3
:1016600003F97480F875300075318C7532E9120316
:1016700092227404F97480F875300075318C7532DB
:10168000EC12043D7980E7A2E0922DA2E1922EA215
:10169000E2922FA2E39214A2E69231A2E709E7A216
:1016A000E09230A2E19232A2E29233A2E39234A21B
:1016B000E69236A2E7923709E7A2E09238A2E292D8
:1016C0003AA2E3923BA2E4923CA2E5923DA2E6A2BA
:1016D000E7923E09E7F5797403F97480F8753000F4
:1016E00075318C7532E912043D7980E7F4F57A0999
:1016F000E7F4F57B09E7F4F57C227980F77401F9CA
:101700007480F875300075318C7532E412039222C2
:101710007401F97480F875300075318C7532E412FB
:10172000043D7980E7227401F9744FF87530007533
:10173000318C7532FC120361227401F9744FF87513
:10174000300075318C7532FC12041822784FE2702B
:10175000067850F208F22275F000303C0475F03C37
:10176000A4AAF075F008A4FBACF0EA75F008A42C6C
:10177000FAC374FD9BFB74FF9A7850F2EB08F222D7
:101780007401F97452F875300075318D753200129C
:101790000361227401F97452F875300075318D754A
:1017A0003200120418227402F9746FF87530007553
:1017B000318C7532FD1204187402F97471F87530A9
:1017C0000075318D753201120418227402F9746F9C
:1017D000F875300075318C7532FD1203617402F9B1
:1017E0007471F875300075318D7532011203612204
:1017F0007401F97455F875300075318C7532F0123A
:1018000003617401F97456F875300075318C7532C6
:10181000F41203617401F97457F875300075318C56
:101820007532F61203617401F97458F87530007559
:10183000318C7532F2120361227401F97455F87516
:10184000300075318C7532F01204187401F9745639
:10185000F875300075318C7532F41204187401F982
:101860007457F875300075318C7532F6120418749F
:1018700001F97458F875300075318C7532F2120424
:1018800018227401F97439F875300075318C75328D
:10189000F81203927401F9743AF875300075318CBE
:1018A0007532FA1203927401F9743BF875300075C1
:1018B000318C7532FB120392227401F97439F87578
:1018C000300075318C7532F812043D7401F9743AA8
:1018D000F875300075318C7532FA12043D7401F9D7
:1018E000743BF875300075318C7532FB12043D2263
:1018F0007402F9741EF875300075318C7532E0127F
:101900000392227402F9741EF875300075318C75DB
:1019100032E012043D22E57C5402600375710378C5
:10192000A17984AA7180021819E7F5F066540F7046
:101930000E18E7C4F5F066540F7004DAEAE422E604
:10194000540FC5F0540FC395F092077401227885A7
:10195000791F7A03E6C4540FF309E6540FF309081C
:10196000DAF2791F78A47A06E6540FF6E366700877
:101970000908DAF4E4C24922792478A97A06C3E393
:10198000961918DAFA9207792478A97A06E3540F9F
:10199000B40F08E6540FB40F108008E6540FB40FCC
:1019A0000B80061819DAE680CB740122C3E396B4E3
:1019B0000902801214600FC3E3F5F0E695F0B40954
:1019C0000280031470E3E9B41F04E4D24922191819
:1019D000E366540F60F080D112194E701D30491A21
:1019E00020301875185085831985821A1209C4751C
:1019F00049B4757D00D245D248E42204227408F926
:101A00007480F875300075318C7532C012043D0257
:101A100019167408F97480F875300075318C7532B8
:101A2000C012043D1219D8227405F97480F875307B
:101A30000075318C7532C0120392227403F97485DB
:101A4000F875300075318C7532C512039222C08250
:101A5000C083E5822420F582E583347DF58374011B
:101A6000F9743CF875300085833185823212043D6B
:101A7000D083D082C082C083E58275F008A4242080
:101A8000F582500205F0A8F0E58375F008A428243B
:101A900000F5837408F97480F8753000858331850A
:101AA000823212043DD083D082124D5922C082C0AE
:101AB00083E58275F008A42420F582500205F0A881
:101AC000F0E58375F008A4282400F5837408F97400
:101AD00098F875300085833185823212043DD083B9
:101AE000D08222C082C083E58275F008A42420F54C
:101AF00082500205F0A8F0E58375F008A4282400C0
:101B0000F5837406F97480F8753000858331858219
:101B10003212043DD083D082227405F97480F875A6
:101B2000300075310075322012043D021916900004
:101B300000121A4E121916223008F3751B00751C7C
:101B40000075689F75690FE568251BC2E0F582E5A1
:101B500069351CF583C082C083E5822400F582E5E7
:101B600083341BF5837402F97480F8753001858322
:101B70003185823212043D78808683088682121A6B
:101B80004E1219167005D0F0D0F022D083D082C347
:101B9000E58313F583E58213F582200714E582457A
:101BA000836022E58224FFF568E58334FFF56980D0
:101BB00007A385821B85831CC3E568951BE5699592
:101BC0001C400280827401223008397410F974803C
:101BD000F87530017531CE75322012043D78987950
:101BE0008075F00AE7B4FF02801AB43C120809D5E8
:101BF000F0F2900FE878C2E2F53C7854F2E4226605
:101C0000540F60E9740122900000121A4E1219D884
:101C10002278A4E6540FB40F03021CAB2008028004
:101C2000E6751B00751C0075689F75690FE56825D2
:101C30001BC2E0F582E569351CF583C082C083E5EF
:101C4000822400F582E583343BF5837402F97480C5
:101C5000F875300185833185823212043D788086A3
:101C600083088682121A4E1219D87005D0F0D0F06F
:101C700022D083D082C3E58313F583E58213F582F6
:101C8000200714E58245836022E58224FFF568E59C
:101C90008334FFF5698007A385821B85831CC3E518
:101CA00068951BE569951C40028082740122789832
:101CB0007A0579ACE6540FC4F5F008E6540F45F008
:101CC000F70809DAEF2275F01E1282E9D5F0FA1250
:101CD00000E475F00F1282E9D5F0FA1200E475F015
:101CE0000F1282E9D5F0FA1200E422120094B2B584
:101CF00075F00F1282E9D5F0FA30B7EF22D216D282
:101D0000A3C256C2A2D259D2A1C258D2A4C257125B
:101D10001CEB121CC6121F63126665120CD1120551
:101D2000C5C2A3C256C2A2C259C2A1C258D2A4C23D
:101D300057126F0D4005C2AF0274D2120094B2B5B3
:101D400075F00F1282E9D5F0FA80E6C2A3C256C23E
:101D5000A2C259C2A1C258D2B775F0021282E9D507
:101D6000F0FA20B744126F0D50028091D216D2A320
:101D7000C256C2A2D259D2A1C258D2A4C257121C72
:101D8000EBD2161266AB401CC2A3C256C2A2C25905
:101D9000C2A1C258D2A4C257121E91126665120C7B
:101DA000D11205C5C2AF0274D2126E98C01D1208BE
:101DB000CED0F0702CC3E51D95F0F57E121E1D12DD
:101DC00015806019D216900000121A4E121E911240
:101DD0006665120CD11205C5B2B5121E1D1213167E
:101DE00022D2A3C256D2A2C259C2A1C258D2A4C200
:101DF00057C216754BFAC2A075F0641282E9D5F08D
:101E0000FA126E93D2A075F0641282E9D5F0FA123C
:101E10006E98D2B712830120B7C7021D651215BF95
:101E2000121672121710A2E0923FA2E19240A2E2B3
:101E300092411217391217931218391218B9121742
:101E4000A67401F974B1F87530017531CE75323070
:101E500012041878B1E2B4FF02E4F27401F974B22A
:101E6000F87530017531CE75323112041878B2E24E
:101E7000B4FF02E4F27404F974D1F87530017531DD
:101E8000CE75323212043D1219031214D112174CBE
:101E900022D216C2A3C256C2A2C259C2A1C258D2ED
:101EA000A4C257C01EC01F78809000007A08E6F0D8
:101EB00008A3DAFA121F6378809000007A08E0F62F
:101EC00008A3DAFA9000001265D4121A28121A3BFD
:101ED000D01FD01E1218F022751E30751F30D21C74
:101EE000C21DC21EC229C22DC22EC22FC214C231AF
:101EF000C230D232C233C234C236C237C238C23A1A
:101F0000C23BC23CC23DC23E757900757A00757B0A
:101F100000757C00786F7422F2087400F278717496
:101F200006F2087400F2C23FC240C241784F740406
:101F3000F278527409F278557401F278567402F20C
:101F400078577404F278587404F2753907753A00BA
:101F5000753B007401785DF2785EF2E408F208F2F5
:101F6000C20822120973121ED81218F01215981204
:101F700015E5C2E0A23F92E0A24092E1A24192E2C6
:101F80001216FA1217261217801217F01218821260
:101F900017CB12152912154E126F6722305B04C23F
:101FA0005B800975F00C20B205D5F0FAD322C3226C
:101FB000E8C0E0E9C0E0EAC0E020043720013412C4
:101FC0001F9C5025755100785EE2600C75F003127D
:101FD00082E9D5F0FA123537785DE2600C75F003CE
:101FE0001282E9D5F0FA123698D0E0FAD0E0F9D0B2
:101FF000E0F82220022220051F3069EDC082C08354
:10200000E57070081278EF400312202F12148A1224
:1020100078BFD083D08280D13069CEC082C083E5C2
:102020007070031220851279C8D083D08280BA30B4
:10203000030C300409D264C263785D02204730018A
:10204000F4D263C264785EE2B40F028013B4100766
:10205000124EFBD251802D75F00384E5F0B40007D9
:10206000124FDED251801DB40107124E76D250803D
:1020700013B40210124DED400B784DE583F208E5E4
:1020800082F2D2522230030C300509D264C2637846
:102090005D02209D3002F4D263C264785EE275F086
:1020A0000384E5F0B400091251914020D251801C04
:1020B000B401091251B94014D25080101251BC40E1
:1020C0000B784DE583F208E582F2D25222D253809A
:1020D00008C25312213F753D00C215D25B754BFA01
:1020E0007440301602740CF548C251C244E5486091
:1020F00039121FB020513375F0031282E9D5F0FA7E
:1021000012027A2016032015183044E120531B7563
:10211000486012115DB40B0D75F0081282E9D5F01C
:10212000FAD251800512213280C3C250D2AF754B12
:10213000FA22533D07F8E53D24A4C8F6053D227870
:10214000A475F00874FFF608D5F0FB223050092082
:102150001B03D21B22C25022C21B22D2538004D2A4
:102160005BC253C215754BFAD21A74403016027412
:102170000CF54812213F753D00C251C250C244C205
:1021800052C25412027A20160320152D121FB020BD
:10219000512920502620522330442D785DE27004CE
:1021A000C244802420531475486012115DB40B1290
:1021B00075F0081282E9D5F0FAD251757D03754B9E
:1021C000FA22757D03122132E54860F23054FD8019
:1021D000B0C0E012234ED0E04021302E0320431B3C
:1021E000205E18C0E0126E9D126E8BD0E0203A097E
:1021F0001282927518101209C4D322203A09128251
:10220000927518201209C4C322D20B7518C0751913
:1022100000751A011209C4302619205D1C20380DE2
:10222000C2AF754CFF754DF8D2AF126E817852E295
:10223000F547222036031222D722E51A543F44C024
:10224000F51A751908C25EC25D205C46126E77D21F
:102250005B803FE51A543F4480F51A751908D25E39
:1022600080E5E51A543F4440F51A751908D25DC25D
:102270005E205C1E126E77D25B8017E51A543F44D5
:1022800000F51A751908D25DC25E8000205C031249
:102290006E8B7518C01209C42230150122C0E0747B
:1022A000108004C0E0741178A4760A0875F00A84DE
:1022B000F608A6F0753D03D0E078ADF2087405F29B
:1022C000D21522C20B754700C2477518C075190098
:1022D000751A021209C422757D00D2457549B4757C
:1022E000185075190F751AFF1209C42275186075F8
:1022F000190F751AFF1209C4C245C2482275187019
:1023000075190F751AFF1209C422126F67E51A5466
:102310003F4400F51A75190B7518C01209C42278CC
:1023200073F208F21238DC7518C0751900751A506E
:102330001209C422400C305C08C25C205D03126E9E
:102340007722205CFC126E9D126E8BD25C221226CC
:1023500085400D122A404008122DFB40031231B96E
:1023600022122690400D122A4B4008122E064003DE
:102370001231C422A290301C01B37859E233F22208
:1023800010760302272E301608C37859E4F202268D
:102390009EE57B541060033043EF7859E260EF0410
:1023A000600302272C201F0320234DD2233008195D
:1023B000C0E0C082C0837400120188D083D082D074
:1023C000E0400302272C0223C97855E224B0401CC8
:1023D000C082C0839025E3E225E00493F5F0E22576
:1023E000E093D083D082C0F0C0E0E222E275189082
:1023F000751909F51A1209C402272C126BF512007F
:10240000D702272C740112220902272C74011221F1
:10241000D140E802272CC2431222EC02272CD270B2
:10242000756F050223EDC0E07401127E0DD0E0024D
:1024300023ED20430320370CC0E07404127E0DD03E
:10244000E00223ED02272C743D0225100223EDC08B
:10245000E0E57C54047005D0E00223EDD0E00227D3
:102460002CC0E0D37401122334D0E00223ED022308
:10247000ED0223ED740012229902272C741012220F
:102480009902272C741112229902272C74201222EF
:102490009902272C7401F97480F875300075318C1D
:1024A0007532F112043D7880E612229902272C74CD
:1024B00001F97480F875300075318C7532F11204B1
:1024C0003D7880E61222A302272C30741C78B2E2F9
:1024D000601778B3F27518C07519097401543F4438
:1024E00080F51A1209C40223FB02272C3074FAE487
:1024F00078B3F27518C07519097401543F4440F55A
:102500001A1209C40223FB751A0112230A0223FBC3
:10251000204308D2431222FD0223FBC2431222ECC5
:102520000223FBE57954106007E412231F0223FB0A
:1025300002272CE5795410600874FF12231F022330
:10254000FB02272C751A0112223A02272C751A0158
:1025500012227B02272C751A0112226202272C7587
:102560001A0112225302272C7400127E0D740112DC
:1025700083350223FB7400127E39740112834402F6
:1025800023FB7400127E5640EC0225687402127E12
:102590000D74011283530223FB7402127E397401FD
:1025A0001283620223FB7402127E5640EC02258CD9
:1025B0007403127E0D74011283710223FB740312E3
:1025C0007E3974011283800223FB7403127E56400D
:1025D000EC0225B030430302251B02272C2043FACE
:1025E000022513272C2404240C241623ED23ED2389
:1025F000ED241E24262432244723ED244C244F248A
:102600006123ED23ED23ED23ED23ED23ED23ED23D6
:10261000ED23ED23ED23ED23ED23ED23ED23ED233A
:10262000ED23ED23ED23ED23ED23ED23ED23ED232A
:10263000ED23ED23ED23ED23ED23ED23ED23ED231A
:10264000ED23ED23ED23ED246E24712474247C24EA
:1026500084248C249424AF24CA24EC250725102537
:102660002325332544254D2556255F2568257525C9
:1026700082258C259925A625B025BD25CA23ED25C3
:10268000D425DD23ED7855E2B40B03A22322C32227
:102690002043097855E2B40D03A22322C322201F50
:1026A0000620230302272CC223300819C0E0C08271
:1026B000C0837400120188D083D082D0E04003022E
:1026C000272C0226C57855E260DAB401061222C32F
:1026D00002272CB4020302272CB40307D243122290
:1026E000FD8049B40908204336303733803EB40AB0
:1026F00002743DB40D0BE57C54047030740D022758
:102700001FB40E0BC37401122334740E02271FC0B2
:10271000E024CED0E05008C0E024B0D0E0500D75E9
:1027200018A0751909F51A1209C48000D27622A2E0
:1027300091301D01B3785AE233F222107603022A57
:10274000E9301608C3785AE4F2022A59E57B54208E
:1027500060033043EF785AE260EF046003022AE737
:10276000201F0320244DD224300819C0E0C082C0AD
:10277000837401120188D083D082D0E04003022A02
:10278000E70227847856E224B0401CC082C08390C0
:10279000299EE225E00493F5F0E225E093D083D072
:1027A00082C0F0C0E0E222E275189075190AF51AAD
:1027B0001209C4022AE7126BF51200D7022AE77445
:1027C00002122209022AE774021221D140E8022AE9
:1027D000E7C2431222EC022AE7D270756F05022786
:1027E000A8C0E07401127E0DD0E00227A8204303A8
:1027F00020370CC0E07404127E0DD0E00227A8023E
:102800002AE7743D0228CB0227A8C0E0E57C5404E7
:102810007005D0E00227A8D0E0022AE7C0E0D37418
:1028200002122334D0E00227A80227A80227A874A6
:1028300000122299022AE77410122299022AE774E0
:1028400011122299022AE77420122299022AE774AF
:1028500001F97480F875300075318C7532F5120409
:102860003D7880E6122299022AE77401F97480F813
:1028700075300075318C7532F512043D7880E612A2
:1028800022A3022AE730741C78B2E2601778B3F210
:102890007518C07519097402543F4480F51A12095D
:1028A000C40227B6022AE73074FAE478B3F2751846
:1028B000C07519097402543F4440F51A1209C40244
:1028C00027B6751A0212230A0227B6204308D243FC
:1028D0001222FD0227B6C2431222EC0227B6E57986
:1028E00054106007E412231F0227B6022AE7E57995
:1028F0005410600874FF12231F0227B6022AE775DE
:102900001A0212223A022AE7751A0212227B022ABE
:10291000E7751A02122262022AE7751A021222537E
:10292000022AE77400127E0D74021283350227B664
:102930007400127E3974021283440227B6740012A6
:102940007E5640EC0229237402127E0D740212831B
:10295000530227B67402127E397402128362022770
:10296000B67402127E5640EC0229477403127E0DA3
:1029700074021283710227B67403127E3974021234
:1029800083800227B67403127E5640EC02296B3016
:1029900043030228D6022AE72043FA0228CE2AE778
:1029A00027BF27C727D127A827A827A827D927E1E6
:1029B00027ED280227A82807280A281C27A827A8C7
:1029C00027A827A827A827A827A827A827A827A88F
:1029D00027A827A827A827A827A827A827A827A87F
:1029E00027A827A827A827A827A827A827A827A86F
:1029F00027A827A827A827A827A827A827A827A85F
:102A000027A82829282C282F2837283F2847284F4F
:102A1000286A288528A728C228CB28DE28EE28FF88
:102A200029082911291A29232930293D2947295400
:102A30002961296B2978298527A8298F299827A812
:102A40007856E2B40B03A22422C32220430978560D
:102A5000E2B40D03A22422C322201F062024030275
:102A60002AE7C224300819C0E0C082C08374011272
:102A70000188D083D082D0E04003022AE7022A8076
:102A80007856E260DAB401061222C3022AE7B402E1
:102A900003022AE7B40307D2431222FD8049B40996
:102AA00008204336303733803EB40A02743DB40DFB
:102AB0000BE57C54047030740D022ADAB40E0BC39B
:102AC0007402122334740E022ADAC0E024CED0E05D
:102AD0005008C0E024B0D0E0500D7518A075190A58
:102AE000F51A1209C48000D27622A292301E01B3D8
:102AF000785BE233F222107603022EA4301608C36C
:102B0000785BE4F2022E14E57B544060033043EF1F
:102B1000785BE260EF046003022EA2201F032025F1
:102B20004DD225300819C0E0C082C0837402120162
:102B300088D083D082D0E04003022EA2022B3F78BF
:102B400057E224B0401CC082C083902D59E225E09A
:102B50000493F5F0E225E093D083D082C0F0C0E08A
:102B6000E222E275189075190CF51A1209C4022EAA
:102B7000A2126BF51200D7022EA2740312220902D0
:102B80002EA274031221D140E8022EA2C2431222C7
:102B9000EC022EA2D270756F05022B63C0E07401A7
:102BA000127E0DD0E0022B6320430320370CC0E0DF
:102BB0007404127E0DD0E0022B63022EA2743D023B
:102BC0002C86022B63C0E0E57C54047005D0E00243
:102BD0002B63D0E0022EA2C0E0D37403122334D0C2
:102BE000E0022B63022B63022B6374001222990212
:102BF0002EA27410122299022EA27411122299028E
:102C00002EA27420122299022EA27401F97480F867
:102C100075300075318C7532F712043D7880E612FC
:102C20002299022EA27401F97480F8753000753172
:102C30008C7532F712043D7880E61222A3022EA290
:102C400030741C78B2E2601778B3F27518C0751949
:102C5000097403543F4480F51A1209C4022B71020F
:102C60002EA23074FAE478B3F27518C0751909749D
:102C700003543F4440F51A1209C4022B71751A031C
:102C800012230A022B71204308D2431222FD022B89
:102C900071C2431222EC022B71E57954106007E4F3
:102CA00012231F022B71022EA2E5795410600874C2
:102CB000FF12231F022B71022EA2751A0312223A51
:102CC000022EA2751A0312227B022EA2751A03127B
:102CD0002262022EA2751A03122253022EA274003F
:102CE000127E0D7403128335022B717400127E392B
:102CF0007403128344022B717400127E5640EC025E
:102D00002CDE7402127E0D7403128353022B717435
:102D100002127E397403128362022B717402127ED6
:102D20005640EC022D027403127E0D74031283715F
:102D3000022B717403127E397403128380022B718B
:102D40007403127E5640EC022D26304303022C9170
:102D5000022EA22043FA022C892EA22B7A2B822B40
:102D60008C2B632B632B632B942B9C2BA82BBD2BC1
:102D7000632BC22BC52BD72B632B632B632B632BAE
:102D8000632B632B632B632B632B632B632B632BD3
:102D9000632B632B632B632B632B632B632B632BC3
:102DA000632B632B632B632B632B632B632B632BB3
:102DB000632B632B632B632B632B632B632BE42B22
:102DC000E72BEA2BF22BFA2C022C0A2C252C402C78
:102DD000622C7D2C862C992CA92CBA2CC32CCC2CA3
:102DE000D52CDE2CEB2CF82D022D0F2D1C2D262D95
:102DF000332D402B632D4A2D532B637857E2B40BB0
:102E000003A22522C3222043097857E2B40D03A26E
:102E10002522C322201F06202503022EA2C2253010
:102E20000819C0E0C082C0837402120188D083D028
:102E300082D0E04003022EA2022E3B7857E260DAF5
:102E4000B401061222C3022EA2B40203022EA2B4BF
:102E50000307D2431222FD8049B4090820433630CB
:102E60003733803EB40A02743DB40D0BE57C540444
:102E70007030740D022E95B40E0BC37403122334FC
:102E8000740E022E95C0E024CED0E05008C0E0249D
:102E9000B0D0E0500D7518A075190CF51A1209C4C0
:102EA0008000D27622A285302901B3785CE233F229
:102EB00022107603023267301608C3785CE4F2020F
:102EC00031D2E57B548060033043EF785CE260EF01
:102ED000046003023265201F03202B4DD22B3008E3
:102EE00019C0E0C082C083740A120188D083D082E6
:102EF000D0E04003023265022EFA7858E224B04056
:102F00001CC082C083903117E225E00493F5F0E203
:102F100025E093D083D082C0F0C0E0E222E27518B1
:102F20009075190DF51A1209C4023265126BF5126B
:102F300000D7023265740412220902326574041249
:102F400021D140E8023265C2431222EC023265D23E
:102F500070756F05022F1EC0E07401127E0DD0E067
:102F6000022F1E20430320370CC0E07404127E0D94
:102F7000D0E0022F1E023265743D023044023265F9
:102F8000022F1EC0E0E57C54047005D0E0022F1E25
:102F9000D0E0023265C0E0D37404122334D0E002E2
:102FA0002F1E022F1E022F1E74001222990232655C
:102FB000741012229902326574111222990232653C
:102FC00074201222990232657401F97480F8753008
:102FD0000075318C7532F312043D7880E612229927
:102FE0000232657401F97480F875300075318C75A2
:102FF00032F312043D7880E61222A3023265307467
:103000001C78B2E2601778B3F27518C075190974AC
:1030100004543F4480F51A1209C4022F2C02326571
:103020003074FAE478B3F27518C075190974045451
:103030003F4440F51A1209C4022F2C751A041223BA
:103040000A022F2C204308D2431222FD022F2CC249
:10305000431222EC022F2CE57954106007E412236E
:103060001F022F2C023265E5795410600874FF129C
:10307000231F022F2C023265751A0412223A0232E3
:1030800065751A0412227B023265751A04122262D7
:10309000023265751A041222530232657400127EE0
:1030A0000D7404128335022F2C7400127E397404BF
:1030B000128344022F2C7400127E5640EC02309C86
:1030C0007402127E0D7404128353022F2C740212A8
:1030D0007E397404128362022F2C7402127E5640D1
:1030E000EC0230C07403127E0D7404128371022F3F
:1030F0002C7403127E397404128380022F2C740303
:10310000127E5640EC0230E430430302304F02326C
:10311000652043FA02304732652F352F3D2F472F68
:103120001E2F1E2F1E2F4F2F572F632F782F1E2F2E
:103130007D2F832F952F1E2F1E2F1E2F1E2F1E2FEC
:103140001E2F1E2F1E2F1E2F1E2F1E2F1E2F1E2F17
:103150001E2F1E2F1E2F1E2F1E2F1E2F1E2F1E2F07
:103160001E2F1E2F1E2F1E2F1E2F1E2F1E2F1E2FF7
:103170001E2F1E2F1E2F1E2F1E2F1E2FA22FA52FDC
:10318000A82FB02FB82FC02FC82FE32FFE3020302C
:103190003B30443057306730783081308A3093305C
:1031A0009C30A930B630C030CD30DA30E430F13068
:1031B000FE2F1E310831112F1E7858E2B40B03A2E6
:1031C0002B22C3222043097858E2B40D03A22B22FC
:1031D000C322201F06202B03023265C22B300819A0
:1031E000C0E0C082C083740A120188D083D082D02C
:1031F000E040030232650231F97858E260DAB40146
:10320000061222C3023265B40203023265B4030718
:10321000D2431222FD804EB4090820433B30373898
:103220008043B40A02743DB40C028039B40D0BE53E
:103230007C54047030740D023258B40E0BC3740405
:10324000122334740E023258C0E024CED0E050086D
:10325000C0E024B0D0E0500D7518A075190DF51A16
:103260001209C48000D27622E5795440601AE57ACA
:1032700054027006122374122380E57A54047006F7
:1032800012272F12273B800C12237412238012273F
:103290002F12273B122AEA122AF6122EA5122EB15D
:1032A000C21F204A0122C24A7518C0751900751A3A
:1032B000541209C422E8C0E07855E264036018782B
:1032C00056E2640360117857E26403600A7858E2BA
:1032D00064036003C38001D3D0E0F82212011430EC
:1032E000080C126865400390FFF11268AA22C052D0
:1032F00012330CD05222300813126865400390FF3D
:10330000F11268AA5005F55212690122E5527005C2
:103310007552108023B41005755211801BB411052D
:103320007552208013B420057552FF800BB4FF0541
:1033300075520080037552FF1269B1E55222C243F3
:1033400075186075190F751AFA1209C4C245C2487A
:1033500022D24375187075190F751AFA1209C42212
:10336000C24375186075190F751AE01209C4C24579
:10337000C24822D24375187075190F751AE01209E8
:10338000C422E4A22692E0A22792E1A22892E2A21D
:103390002C92E3F5747575051238527403500412BB
:1033A00039D8221239B27891E6C0E0E57A54026049
:1033B00012D0E0C0E054071233E0D0E0C0E0540780
:1033C0001233E0E57A54046014D0E0C0E0C454073E
:1033D000123405D0E0C0E0C45407123405D0E02216
:1033E000A223301C01B34007D320E10A023404C3F6
:1033F00020E203023404301C01B3E4500114785974
:10340000F212238022A224301D01B34007D320E111
:103410000A023429C320E203023429301D01B3E437
:10342000500114785AF212273B22B40207205107A8
:10343000C250C2520234B8C082C08390EA60E53DF7
:10344000606324FB405F78A4E6540F758300F58227
:10345000D53D02805075F00AA4F58275830008E618
:10346000540F2582F582D53D02803AE58275F00A37
:10347000A4F58285F08308E62582F5825002058353
:10348000D53D028020E58275F00AA4F582C0F0E502
:103490008375F00AA4D0F025F0F58308E62582F5BF
:1034A0008250020583784DE583F208E582F2C2512D
:1034B000C250D252D083D08222C289C28BD293C250
:1034C000B422C0F075F0FAD5F0FD75F064D5F0FDCA
:1034D000D0F0221234C21234C21234C21234C212D8
:1034E00034C21234C222D293C2B475F005128301E1
:1034F00020B20612830130B203D5F0F1128301220B
:10350000C0F075F008A2E7B392B4C2931234C2C2FD
:10351000B4D2931234C2C0E0E430B201040030B23D
:1035200001040030B20104D36003D5E001C3D0E050
:1035300033D5F0D1D0F022D293C2B4D2B21234C279
:10354000C2931234D3D2931234D320160330641CA6
:1035500078907601087480F608A2A3B392E4F6741A
:103560009008F608F608F608F60235AC789076036F
:10357000087680087480A25692E5A2A3B392E42054
:103580001608A25992E1A22692E0F608748020164D
:103590001220640FE55154074480A25892E5A2A17D
:1035A000B392E4F6087480F608F608F675F007782A
:1035B000907E007F00E62EFEE6123500F62FFF0813
:1035C000D5F0F2EED333123500F8EFD333687064E0
:1035D0007890B6FF5F0561E56124FE5014756102C5
:1035E00020180ED2187518C0751900751A03120923
:1035F000C4201608785EE2600330640302369478D3
:1036000096E620E35920E24920E1277891E6B600CA
:103610002108B6420908E6D263123AE48076B6552C
:103620001108B6000D08794DE6F30809E6F3D25209
:10363000D2638060E5616017D56114301811C2183B
:103640007518C0751900751A041209C4757F0380B6
:10365000437891863D08D25179A47A04800B789101
:10366000D25075710579987A05D26375F00FE6C46A
:10367000540FF755F0F5F009E6540FF755F0F5F053
:103680000908DAEAE5F0B40F051977EEC250785E62
:10369000E212342A1234E622D293C2B4D2B21234E5
:1036A000C2C2931234D3D2931234D320161F306384
:1036B0002378907611087480F608A2A3B392E4F6FA
:1036C000749008F608F608F608F602371D7890762A
:1036D000150236D878907613087680087480A25642
:1036E00092E5A2A3B392E4206314A25792E1A2A4AC
:1036F000B392E0201608A25992E1A22692E0F608C1
:10370000748020630FE55154074480A25892E5A2CB
:10371000A1B392E4F6087480F608F608F675F0078F
:1037200078907E007F00E62EFEE6123500F62FFF31
:1037300008D5F0F2EED333123500F8EFD3336870CA
:10374000627890B6FF5D0560E56024FE50147560F8
:103750000220190ED2197518C0751900751A0512B4
:1037600009C4785DE2600330630302380E7896E6A0
:1037700020E36520E25520E1487891E6B600220872
:10378000B6420A08E6D264123AE402380EB655117F
:1037900008B6000D08794DE6F30809E6F3D252D2D7
:1037A00064806BE5606017D56014301911C219751B
:1037B00018C0751900751A061209C4757F030238FE
:1037C0000ED26478918640D24480437891863D0839
:1037D000D25179A47A04800B7891D2507571057911
:1037E000987A05D26475F00FE6C4540FF755F0F5DA
:1037F000F009E6540FF755F0F5F00908DAEAE5F0BC
:10380000B40F051977EEC250785DE212342A1234F3
:10381000E622785EE2601024FD400C75F00312820F
:10382000E9D5F0FA12353722785DE2601024FD40C8
:103830000C75F0031282E9D5F0FA12369822C0E036
:1038400030630C7518B0751900751A001209C4D0D0
:10385000E022D293C2B4D2B21234C2C2931234D391
:10386000D2931234D37890E575540FC44407F60808
:10387000E57423A2E392E5A2E292E3542AD2E7F6AA
:1038800008E574A2E392E1A2E492E3542AD2E7F6B7
:1038900008E574A2E692E1A2E792E3540AD2E7F6C1
:1038A000748008F608F608F675F00778907E007FB9
:1038B00000E62EFEE6123500F62FFF08D5F0F2EEF8
:1038C000D333123500F8EFD33368700B7890B6FF1E
:1038D000061234E6C380041234E6D32275750878E4
:1038E00073E2F574123852740040051239B2800345
:1038F0001239D87575097874E2F57412385274016A
:1039000040051239B280031239D82222E5795420B9
:1039100060F97575047574FF123852740250041200
:1039200039D8221239B278937948E6F30809E6F3D8
:1039300008794AE6F30809E6F37891E6A2E092E214
:103940005414F5F008E623A2E592E0540345F0F59F
:10395000F0784CE265F0C0E0E5F0F2D0E030E21F34
:10396000C0E0C0F0E5F075F04930E20375F04A754B
:1039700018C075190085F01A1209C4D0F0D0E054AF
:103980000370030239B1E5F05403B4030575F04840
:103990008013B4020575F047800BB4000575F04B39
:1039A000800375F04C7518C075190085F01A12095E
:1039B000C422F5F02442F8E2B40205227402F22295
:1039C00050FA7402F2E5F02432F5F07518C075195A
:1039D0000085F01A1209C422F5F02442F8E2601AB8
:1039E000D5E016F2E5F0243CF5F07518C075190025
:1039F00085F01A1209C4757F03F222D293C2B4D2A1
:103A0000B21234C2C2931234D3D2931234D3789008
:103A1000E575540FC44403F6087680087480A256F6
:103A200092E5A2A3B392E4A25992E1A22692E0F613
:103A3000087480A25892E5A2A1B392E4F6087480BB
:103A4000F608F608F675F00778907E007F00E62EFF
:103A5000FEE6123500F62FFF08D5F0F2EED3331252
:103A60003500F8EFD3336870717890B6FF6C7896B4
:103A7000E620E33020E22020E1607891E6B6005AAB
:103A800008B6551108B6005208794DE6F30809E664
:103A9000F3D252804A80437891863D08D25179A46E
:103AA0007A04800B7891D25075710579987A0575F2
:103AB000F00FE6C4540FF755F0F5F009E6540FF790
:103AC00055F0F5F00908DAEAE5F0B40F051977EEDC
:103AD000C2507864E212342A80051234E6D32212EE
:103AE00034E6C322B4FF15D270756F0512383E75E7
:103AF00018C0751900751A071209C422B4BC030254
:103B00003B15B4BD03023B47B4BE03023B79B4BFCF
:103B100003023BAB222063147408F97480F87530FB
:103B2000017531CE75324012043D80127408F9746B
:103B300080F87530017531CE75324812043D74112C
:103B40007888F6123BDD222063147408F97480F83B
:103B50007530017531CE75325012043D80127408F3
:103B6000F97480F87530017531CE75325812043D04
:103B700074127888F6123BDD222063147408F974FD
:103B800080F87530017531CE75326012043D8012B7
:103B90007408F97480F87530017531CE7532681289
:103BA000043D74137888F6123BDD222063147408F8
:103BB000F97480F87530017531CE75327012043D9C
:103BC00080127408F97480F87530017531CE753241
:103BD0007812043D74147888F6123BDD227881E671
:103BE0001201584004741ED3227882E61201A840C4
:103BF0000C741FD322126BF51200D7C3227880E613
:103C000060F9B4FF08D270756F05023DFFB402126F
:103C1000203A0312383E7888E61221D1400280DB38
:103C200080D3B4090CC0E07404127E0DD0E0023DD4
:103C3000FFB438087883E6123E1080BFB4390878A4
:103C400083E6123E1A80B4B43A2530742012383E0E
:103C500078B2E278B3F2788886F07518C0751909E1
:103C6000E5F0543F4480F51A1209C48088808CB472
:103C70003B223074F812383EE478B3F2788886F04C
:103C80007518C0751909E5F0543F4440F51A12093A
:103C9000C4023BF5B43C0D12383E7888861A1223D4
:103CA0000A023BF5B43D2B12383E204311D2437536
:103CB000187075190F751AE91209C4023BF5C24351
:103CC00075186075190F751AE91209C412528D0220
:103CD0003BF5B43E13E5795410600A12383EE41205
:103CE0003E1F023BF5023BFBB43F14E579541060E4
:103CF0000B12383E74FF123E1F023BF5023BFBB431
:103D0000400D12383E7888861A12223A023BF5B4EA
:103D1000410D12383E7888861A12227B023BF5B498
:103D2000420D12383E7888861A122262023BF5B4A0
:103D3000430D12383E7888861A122253023BF5B49E
:103D4000440E7400127E0D7888E6128335023BF52E
:103D5000B4450E7400127E397888E6128344023B23
:103D6000F5B446097400127E5640E880D5B4470E7B
:103D70007402127E0D7888E6128353023BF5B44834
:103D80000E7402127E397888E6128362023BF5B423
:103D900049097402127E5640E880D5B44A0E740375
:103DA000127E0D7888E6128371023BF5B44B0E74D7
:103DB00003127E397888E6128380023BF5B44C0901
:103DC0007403127E5640E880D5B44D1812838F7864
:103DD00088E6543F4480F51A75190B7518C012090E
:103DE000C4023BF5B44E0C30430612383E023CBED2
:103DF000023BF5B44F092043F712383E023CAD12A6
:103E0000383E7518C0751907F51A1209C4023BFB34
:103E10001222997888E678AEF2221222A380F478F2
:103E200073F208F21238DC7888E6543F44C0F51A81
:103E300075190B7518C00209C4700575631E8002E0
:103E4000D21122C298C299322016F830991EC29916
:103E5000204F057535008014C0F0C0E0C0D075D08B
:103E600010E535124173D0D0D0E0D0F02098013267
:103E7000C298204FFAC0F0C0E0C0D075D010304ECC
:103E800005C24E754100E54524FE4003754502E537
:103E90004120E71FE5415407232435C0E074003476
:103EA00040C0E0E5992205412544F544D0D0D0E05A
:103EB000D0F032543F23232436C0E07400343FC096
:103EC000E0E59922156280DE80DCD562FBB5441204
:103ED000D20FE8C0E078A974FAF2D0E0F87541009A
:103EE00080CA024045B462FA80BC80BAB42AF3802A
:103EF000B5F56224C6E56240E924F5E56250E305C4
:103F00006280A37818F21562809C7819F21562809D
:103F100095781AF21562808E781BF2156280877888
:103F20001CF215628080781DF21562023EA6781E92
:103F3000F21562023EA602405D00023EE500023E2E
:103F4000EA00023EEC00023EF100023EC400023EE6
:103F5000C400023EC400023EC400023F0300023F10
:103F60000A00023F1100023F1800023F1F00023FFB
:103F70002600023F2E00023ECA00023ECA00023E58
:103F8000CA00023ECA00023ECA00023ECA00023E09
:103F9000CA00023ECA00023ECA00023ECA00023EF9
:103FA000CA00023ECA00023ECA00023ECA00023EE9
:103FB000CA00023ECA00023ECA00023ECA00023ED9
:103FC000CA00023ECA00023ECA00023ECA00023EC9
:103FD000CA00023ECA00023ECA00023ECA00023EB9
:103FE000CA00023ECA00023ECA00023ECA00023EA9
:103FF000CA00023ECA00023ECA00023ECA00023E99
:10400000CA00023ECA00023ECA00023ECA00023E88
:10401000CA00023ECA00023ECA00023ECA00023E78
:10402000CA00023ECA00023ECA00023ECA00023E68
:10403000CA0002405D800E802D803180358038803E
:104040003B80488046B40909754400754100023E32
:10405000A6B44209754400754180023EA67544002D
:10406000754100023EACB51EDC023EA6B51FD6026D
:104070003EA6F542023EA6F543023EA6B544C675ED
:10408000452012408D754100023EAC80D0854237FC
:10409000127329D24FE537B4460302596EB4470470
:1040A00012733F22B4500E854336127304C2ACC261
:1040B0004F75730722B45312854336E543700A12D5
:1040C0007304C2ACC24F75730222B4540E854336DA
:1040D000127304C2ACC24F75730122B4550E8543EE
:1040E00036127304C2ACC24F75730322B4560E85E8
:1040F0004336127304C2ACC24F75730422B4570E18
:10410000854336127304C2ACC24F75730522B4588E
:104110000E854336127304C2ACC24F75730622B4C7
:104120004E3D854336E543B4000B127304C2ACC266
:104130004F75730822B4010B127304C2ACC24F75E1
:10414000730922B4020B127304C2ACC24F75730E12
:1041500022B4030B127304C2ACC24F75730F222436
:10416000BF24E6400485433622C24F22C538253895
:10417000C53822E53524F0400EE535232492C0E011
:1041800074003441C0E022759906C24F753500D2E3
:10419000B622802F8034803680388039803E804639
:1041A00080488051804F804D804B80468050800EEB
:1041B00002423A753503F59912416C053522E53610
:1041C0000241E8753800740380ECE51E80E8E51FC5
:1041D00080E402429EE53875350F80DA120A021239
:1041E0003E39883680D0E53680C9E536A24392E074
:1041F00080C1753503A8360536E676FF80B8E5360A
:10420000C313603214700BA22392E0B392E1440412
:1042100080D614700BA22492E0B392E1440880C8C7
:10422000147008A22592E0440C80BD147008A22BE3
:1042300092E0440C80B274FC80AEE53614702574B4
:1042400008305C12305D044406809D305E044403F7
:10425000809644078092A25D92E0A25E92E1A2263F
:1042600092E280841470157410A22392E0A224922A
:10427000E1A22592E2A22B92E30241E814700D74B0
:1042800018A21892E0A21992E10241E814700BA260
:104290005F92E0A26192E20241E8E40241E8E53780
:1042A000B441067535040241B6B44212E5366003E6
:1042B000301103120A1A75631E74420241B3B444EA
:1042C0000280F8B44B028003024363E53654F8B42D
:1042D000083EE5365407700B751A1912223AE53775
:1042E000024398B4010B751A19122253E5370243A1
:1042F00098B4020B751A19122262E537024398B47A
:10430000030B751A1912227BE53702439802418785
:10431000B42003024187B42826E53620E008304364
:104320000B12528D8006204303127550E536A2E031
:104330009243756E015003756E02E5370241B3B4C6
:10434000300CE53654F8127E0DE5370241B3B4382F
:104350000CE53654F8127E39E5370241B302418745
:10436000024187B4430FB5360375460375350775AB
:1043700036AC0241B6B44A26E536701F205E1C20DA
:104380005C087419126E9D126E8B75181075190FDA
:10439000751AF01209C4E5370241B3024187B445EA
:1043A000067535060241B6B4510675350C0241B6A4
:1043B000B44D0EE53612811DE5375002B2E70242D8
:1043C000BBB44C0675350E0241B6B4460280C9B482
:1043D000470280C4B44F08C245C246C24780B9B440
:1043E000590FE536700B857E36745975350D0241CF
:1043F000B6024187E573B4000122B40717C2AC12BC
:104400008319128319D29912716FC24FD2B61273E7
:1044100004024518B40117C2AC128319128319D2D1
:1044200099120FC6C24FD2B6127304024518B403D4
:1044300017C2AC128319128319D29912104BC24FB2
:10444000D2B6127304024518B40217C2AC12831913
:10445000128319D299120EE7C24FD2B61273040218
:104460004518B40417C2AC128319128319D29912D9
:104470000F29C24FD2B6127304024518B40517C2F1
:10448000AC128319128319D2991202ACC24FD2B660
:10449000127304024518B40617C2AC1283191283B2
:1044A00019D299121093C24FD2B612730402451852
:1044B000B40817C2AC128319128319D299126D3540
:1044C000C24FD2B6127304024518B40917C2AC1217
:1044D0008319128319D299126CB9C24FD2B61273D2
:1044E00004024518B40E17C2AC128319128319D2F4
:1044F00099126DC2C24FD2B6127304024518B40F9E
:1045000017C2AC128319128319D299126E04C24FCA
:10451000D2B612730402451875730022E565C267AE
:104520006002D267E552F553C24820520C20501B5E
:10453000305103024651024B1C120102784DE2F544
:104540008308E2F582121A4E02470E120102121C73
:10455000AE121B386017121BC8603C12383E75182B
:104560002075190F751AEC1209C402459A206305CB
:10457000205F0A8003206105124BC8501AC082C018
:10458000831200E41220D1D083D08230510CE53D5B
:1045900060081219D8700302470E754A3CD54617B9
:1045A0007518C0751900751A531209C4754603753C
:1045B0007D00D2467549B4024B09D270756F051261
:1045C000383E7518C0751900751A071209C475515F
:1045D0000412381212382875F06412011E024B1CA6
:1045E000206324E57B540860CE300818C0E0C08208
:1045F000C0837411120188D083D082D0E040028041
:10460000B9024628024628E57A548060AA30081884
:10461000C0E0C082C0837410120188D083D082D0E1
:10462000E04002809502462812234E401E205E156F
:10463000302E03204309900FE9124B25024B1C1228
:104640004AA6024B1C124AAC024B1C124AB2024B45
:104650001C120102E53D608878A4E6B40A03025208
:104660007F121C11707D206305205F508003206144
:104670004B124BC84046206325300819C0E0C08269
:10468000C0837413120188D083D082D0E04003022B
:10469000470E02469802470E124A8202459A300897
:1046A00018C0E0C082C0837412120188D083D08207
:1046B000D0E0400302470E80DF02470E1200E4C044
:1046C00082C08312215FD083D082305013C082C059
:1046D00083120102121CAED083D082121916602EF2
:1046E00002459A785D206402785EE2B40F0A124EA9
:1046F000B3C251D25002454EB4100280F112383E7E
:1047000075182075190F751AEB1209C480D2306321
:1047100030300819C0E0C082C083740C120188D008
:1047200083D082D0E0400302474102472D757502D5
:10473000785FE27864F212149612502C500302450E
:104740009A306430300819C0E0C082C083740D1202
:104750000188D083D082D0E04003024774024760D2
:104760007575037860E27864F21214A212502C502E
:104770000302459A1274FF40031234B9E53C0470F9
:104780000302459A754A00754603C247C24620484F
:1047900002C245C082C083124C6FD083D0825006C3
:1047A000124AC1024B1CC082C0831205DBD083D0E9
:1047B000825006124AC1024B1CE58224CEE58334A6
:1047C000FF5017124BB64012C212C2131232B5502C
:1047D00006124AB2024B1C0249BD12234E5012125D
:1047E0004AB2024961124AAC024961124AA6024920
:1047F00061205EF1302E032043F13063037854E2F0
:10480000306402E53C120158400302481602485A3F
:10481000124AA00249613008F73014F4303DF11219
:1048200051834036A263303E01B3502E300818C089
:10483000E0C082C0837409120188D083D082D0E0A6
:10484000400280CC024847C082C0831270FBD083F4
:10485000D0825006124AB7024961301425D239304D
:104860000819C0E0C082C0837414120188D083D0BC
:1048700082D0E0400302487D02487BC23912518356
:1048800050030248F21270A7A2E09212A2E1921322
:10489000A263303E01B3C0E09206501E1271515027
:1048A0001930390EE4A21292E0A21392E1B402028E
:1048B0008008D0E0124A8E024961D0E0B4000520A1
:1048C0000622802BB4012220061A7518C075190023
:1048D000751A091209C4203906124ABC024961122C
:1048E0004B79800E126FFA8009B402ED2006DB12BC
:1048F00070523008581251834053300819C0E0C03C
:1049000082C0837408120188D083D082D0E0400333
:1049100002494D02491620671AA263926685836692
:10492000858267124B75C263C2641200F875650216
:10493000024B1C756500E5836566F5F0E5826567E9
:1049400045F07006124AC6024961125220124B25E8
:10495000E5795410600BC082C083124D7FD083D0A4
:1049600082124BBF5009124D5930E103024B1C1209
:1049700032B540F8C2A1D258D2A4C2577551001224
:104980003812123828121A4EC082C08312215FD00A
:1049900083D08220520920501720511C024B1C1238
:1049A0000102784DE2B5830D08E2B582080249BDE7
:1049B0001219166008024B091219D870F830142425
:1049C000E4A21292E0A21392E1B4030512707E8079
:1049D00013B40205126FFA800BB4010512705280F5
:1049E00003126FD1300819C0E0C082C08374061270
:1049F0000188D083D082D0E04003024B09024A00F4
:104A0000E57954016022E5824583601C30630378B8
:104A100054E2306402E53C1201584003024A22028B
:104A20004A28124A94024B1C122361500F124A9AD0
:104A300075F01E12011E1200C1024B1CB243123847
:104A40003E30431D75187085831985821A1209C47A
:104A5000C2A3C256D2A1C258D2A4C2571275508066
:104A60001B75186085831985821A1209C4D2A3C2E6
:104A700056D2A1C258C2A4C25712528D1200D702F8
:104A80004B1C126BEB024AC9126BEB024AC9126B48
:104A9000EB024AC9126BEB024AC9126BEB024AC91C
:104AA000126BEB024AC9126BEB024AC9126BEB02A2
:104AB0004AC9126BEB8012126BEB800D126BEB800C
:104AC00008126BEB8003126BEB7565007566FF7562
:104AD00067FFD27712383E75182085831985821AB0
:104AE0001209C41200C1C27722E57A54087003206B
:104AF0006316E552046011146564600C7518C07586
:104B0000190185521A1209C422126BEBD2771200D6
:104B1000ABC2777565007566FF7567FFC251C250FD
:104B2000E553F5522230430EC2A3C256C2A2C25967
:104B3000D2A4C257800CD2A3C256C2A2C259C2A4E8
:104B4000C257A263920AD209126BEB741C126E9DBB
:104B5000126E8BE5795440600620A803123382124E
:104B6000383E124AE975181085831985821A120990
:104B7000C41200D722126BEB22126BEB75F03212CB
:104B8000011E227408F97480F875300175310375BF
:104B9000329012043D7885E60856085604601412D7
:104BA00000E41220D1305109E53D60051219D860AA
:104BB00002C322D32222E582249CE58334FF22E52E
:104BC00082249CE58334FF22A240E5824583601065
:104BD000E582249CE58334FF5004A23F8002A24179
:104BE00022E5822582F582E5833583F583E58225FA
:104BF00082F582E5833583F583E5822400F582E53D
:104C000083345BF5837404F97400F875300185838F
:104C100031858232120418227885E654C0F58378F3
:104C200086E630E402240A2323543C4583F5837846
:104C300085E6C4540375F00AA4F5F0E6540F25F098
:104C4000030303F5F053F0E085F08254034583F548
:104C5000837884E6C4540375F00AA4F5F0E6540F93
:104C600025F04582F58222C39582E5F095832212D4
:104C700051835003024CF7124BE17800E2B4FF037A
:104C8000024CF71277CC124C187880A68308A682C3
:104C90007800E2F58308E2F58208E2F5F008E21216
:104CA0004C67502B7800E2F58308E2F58278808625
:104CB000F008E6124C6750417802E2F58308E2F50D
:104CC00082788086F008E6124C67402D024CF77817
:104CD00000E2F58308E2F582788086F008E6124C5F
:104CE0006740167802E2F58308E2F582788086F064
:104CF00008E6124C675002C322D322C3E58233F583
:104D000082E58333F583E5822400F582E583349AD6
:104D1000F5837402F97453F8753001858331858207
:104D20003212041822C3E58233F582E58333F5831A
:104D3000E5822400F582E583349AF5837402F974E0
:104D400053F87530018583318582321203612278F0
:104D5000537400F208E4F2801E3008F3C082C0836E
:104D6000124CFBD083D082E5822418E58334FC40CA
:104D7000067853E24402F27854E2F5F018E222E5B4
:104D8000822400F582E58334BAF5837401F97480D6
:104D9000F875300185833185823212043D7880E6D2
:104DA00060422323C0E05403F5F0D0E054FC24001B
:104DB000F582E5F034CAF5837404F97480F875302F
:104DC0000185833185823212043D7880E60886F0C1
:104DD0007873F208E5F0F275F0021282E9D5F0FA84
:104DE0001238DC2274FF7873F208F280EAE572B4BC
:104DF000220575F0048013B42A0575F006800BB403
:104E0000420575F00C800375F002782EE2540F70A5
:104E10004F08D5F0F7E2540F75F00AA4F5827583B8
:104E20000008E2540F2582F582E58275F00AA4F5A8
:104E30008285F08308E22582F58250020583E582AF
:104E400075F00AA4F582C0F0E58375F00AA4D0F0ED
:104E500025F0F58308E22582F58250020583C322FE
:104E6000D322782EE2600BF5F008E2240A4005D543
:104E7000F0F7C322D322782EE572B4220A757104AA
:104E8000799A75F0088024B42A0A757105799875A5
:104E9000F00A8017B4420C757105799875F00A789C
:104EA000348008757103799C75F006E2F70809D51E
:104EB000F0F922C082C08378989002E075F00AE091
:104EC000F608A3D5F0F99002EAE0F571D083D0821C
:104ED00022C082C08378989002E075F00AE6F0085C
:104EE000A3D5F0F9E5719002EAF0D083D0822212C6
:104EF0004E7612191622D083D08222124E76124E8E
:104F0000D112213FC082C083753D01782EE2540F3B
:104F100070E408E2540F70DE08E2540FC4F5F008A4
:104F2000E2540F45F0F58308E2540FC4F5F008E2AF
:104F3000540F45F0F582C26D78A47900C3E58294E0
:104F400010F582E5839427F58340030980EEE5821E
:104F50002410F582E5833427F583E96004D26DF6E9
:104F6000087900C3E58294E8F582E5839403F5832C
:104F700040030980EEE58224E8F582E5833403F5F9
:104F800083E9206D046004D26DF6087900C3E582E0
:104F90009464F582E5839400F58340030980EEE58F
:104FA000822464F582E5833400F583E9206D046092
:104FB00004D26DF608E58275F00A84206D02600265
:104FC000F608E5F0F6E8245DF53DD083D08222793D
:104FD000A477000975F00577FF09D5F0FA22124E83
:104FE00076124ED1124FCF75F008E572B4220478D4
:104FF0002E8013B42A047830800CB44204783680B2
:1050000005782E75F006753D06E2540F700608D53A
:10501000F0F7800979A4E2F70809D5F0F922124FD8
:10502000DE1219D822124EFB1219D8227864E270CF
:10503000030250E124FD4038C082C0831200E41214
:10504000513DD083D08220521620510B3050361261
:10505000191670310250E11219D870290250E17806
:105060004DE2B5832008E2B5821B6582701780711E
:10507000E224E24070C082C0831200E4127991D031
:1050800083D08250030250E37864E2B40F0C1250D4
:105090001E604E124EEF604980EBB410071250258F
:1050A000603F80E175F00384E5F0B4000712501E04
:1050B00070D3802DB40107124EEF70C98023B40263
:1050C0001EC082C083124DEDE5828583F0D083D06F
:1050D0008240B2658270AEE5F0658370A880028080
:1050E000A4C322D322C082C0831200E41279E7D085
:1050F00083D0825002D3227864E275F00384E5F015
:10510000B4000A1251911219D870EA802CB4010A25
:105110001251B912191670DD801FB4021EC082C070
:10512000831251BCE5828583F0D083D08240C6656E
:105130008270C2E5F0658370BCC32280B8754832C6
:10514000D25B305409C254C07512027AD075E5485A
:10515000D36018C252C251C250121F9C50E412397F
:10516000FB2052062051033050D8C3C0D0A875741C
:1051700005B802027404D0D040051239B28003127F
:1051800039D822E582B4E807E583B40F02D322C3FD
:1051900022124E625002D322782EE260F9F5F00816
:1051A000753D06E2540F700608D5F0F7800979A422
:1051B000E2F70809D5F0F9C322027B09124E6250CA
:1051C00004D322C322782EE20860F6B40108E2F587
:1051D0008275830080EDB40212E275F00AA4F582B4
:1051E00008E22582F58275830080D8B40320E27539
:1051F000F00AA4F58208E2258275F00AA4F58285FA
:10520000F08308E22582F58250B9058380B5B404A5
:1052100005782F024E15C39404F5F0782F024E0C3A
:10522000B263B264755107123812123828B264B2F0
:10523000637518C0751900751A0C1209C430660C14
:105240007518B0751900751A001209C4124AE9756B
:10525000181085661985671A1209C422E53DB40342
:105260001C78A4E6B40A1608E624F6401008E624E2
:10527000F6400A18E675F00AA40826C322D32212C3
:10528000525C500302466178ACF20252DC12755057
:1052900012838FC245C2482253335355539153BD95
:1052A00053D453EB5402541954285437544654558C
:1052B000548954B154B954CB54DA551655655588B0
:1052C000559F55C055DC55F856045620563C564857
:1052D00056645680568C56A55307530778ACE22483
:1052E000E040241257EE401378ACE225E0049052DF
:1052F0009893C0E0E225E093C0E0220258A612583D
:10530000A51200D7024B1C740A0258A6D2A1C2589B
:10531000C2A4D2571258A41200E412215F205102F5
:10532000D322E53DB402F978A4E624F640F208E67B
:1053300024F6221258A312530C401578A4E6243008
:10534000F51E08E62430F51F1218F012666580AECF
:1053500074200258A61258A312578D402F1277CCF2
:1053600078A4E6C40846F5F078A8E654030303459C
:10537000F07885F678A6E6C40846F5F078A9E6C484
:105380002345F07886F61277AD0252FE741E02585D
:10539000A61258A312573E401F1277CC78A4E6C439
:1053A00008467884F678A6E6C408467883F6E4785A
:1053B00082F61277AD0252FE741F0258A61258A34D
:1053C0001258877518C0751900751A0F1209C4D2C2
:1053D0005F0252FE1258A31258877518C075190043
:1053E000751A101209C4C25F0252FE1258A3125855
:1053F000877518C0751900751A511209C4D2610257
:1054000052FE1258A31258877518C0751900751AE4
:10541000521209C4C2610252FE1258A31258877573
:105420001A1B12223A0252FE1258A3125887751AFA
:105430001B1222530252FE1258A3125887751A1BD0
:1054400012227B0252FE1258A3125887751A1B12A1
:1054500022620252FE1258A31232B5402712588718
:1054600012755012838FC245C248C243784DE2F58F
:105470008308E2F58275186085831985821A1209FE
:10548000C40252FE74160258A61258A31232B54036
:10549000F3125887127550D243784DE2F58308E233
:1054A000F58275187085831985821A1209C4025213
:1054B000FE1258A320439E80D01258A3125887751D
:1054C000F0C81282E9D5F0FA0274D21258A3125829
:1054D00087751A1B12230A0252FE1258A320150DBB
:1054E000125706402C1258B9402778ADF278ADE239
:1054F000F552F5531258877518C085521A7519035D
:105500003015037519021209C40252FE74190258AB
:10551000A6741A0258A61258A320150D1257064059
:10552000F01258B940EB78ADF278ADE2F55212586E
:10553000877518C085521A75190630150375190537
:105540001209C4126902124BB5D2A2C259C2A1D229
:10555000581200E412215F741820500620510330C5
:1055600052B102452A1258A330742D78B2E278B3B2
:10557000F21258877518C0751909741B543F44807E
:10558000F51A1209C40252FE1258A330740A1257B7
:1055900006500A741C0258A6741D0258A670CF1239
:1055A00058A33074F3E478B3F21258877518C075B5
:1055B0001909741B543F4440F51A1209C40252FEE3
:1055C0001258A37400127E0D7518C075190A741B49
:1055D000543F4400F51A1209C40252FE1258A37433
:1055E00000127E397518C075190A741B543F448027
:1055F000F51A1209C40252FE1258A37400127E5604
:1056000040DD80BF1258A37402127E0D7518C0755C
:10561000190C741B543F4400F51A1209C40252FEBF
:105620001258A37402127E397518C075190C741BB8
:10563000543F4440F51A1209C40252FE1258A37492
:1056400002127E5640DD80BF1258A37403127E0DF5
:105650007518C075190C741B543F4480F51A120953
:10566000C40252FE1258A37403127E397518C07515
:10567000190C741B543F44C0F51A1209C40252FE9F
:105680001258A37403127E5640DD80BF7404127E4C
:105690000D7518C075190B741B543F4440F51A1250
:1056A00009C40252FE12838F7518C075190B741B42
:1056B000543F4480F51A1209C40252FEC2A1D258C6
:1056C000C2A4D257124BB51200E412215F20520837
:1056D00020501C205129D322784DE2F58308E2F5B1
:1056E00082120102300806124D5920E2E9C322124B
:1056F0001B3870E2784DE583F208E582F280E21211
:105700001C1170D280EED2A1C258C2A4D257125836
:10571000A41200E412215F205102D322E53D60FA79
:1057200024FC40F6A93D78A47A00EA75F00AA42684
:1057300040E8C5F070E4AAF008D9EFEAC322D2A18C
:10574000C258C2A4D2571258A41200E412215F20FA
:105750005102D322E53DB404F9F5F078A4E624F62D
:1057600040F008D5F0F778A4E675F00AA4082624DE
:10577000E8402E78A6E675F00AA4082624C4402145
:1057800022E0E2E0E1E0E1E0E0E1E0E1E0D2A1C23C
:1057900058C2A4D2571258A41200E412215F20511B
:1057A00002D322E53DB406F9F5F078A4E624F640EC
:1057B000F008D5F0F778A6E675F00AA4082660E1AF
:1057C000C0E024F3D0E040D990578093F978A4E664
:1057D00075F00AA4082660C9C0E029D0E040C2786C
:1057E000A8E624F640BB78A9E624F940B4223008A4
:1057F0007C784D740FF20874E9F220157C78ACE2E5
:105800002400F5827583D07401F97480F875300135
:1058100085833185823212043D7880E6120158502A
:105820006278ACE22400F5827583D17401F974804A
:10583000F875300185833185823212043D7880E627
:105840001201A8503678ACE22400F5827583CF743B
:1058500001F97480F8753001858331858232120434
:105860003D7880E620630C20E01530E10C1256BC38
:10587000740D2220E20920E3F4C322740E80067422
:105880000C8002740BD32220151812383E784DE29A
:10589000F58308E2F5827518E085831985821A126E
:1058A00009C422222222C0E0126BEB1258A3D0E0DE
:1058B0001267E21200AB024B1CC052C082C083F5DB
:1058C00052126865D083D082E552D052B322C538D7
:1058D0002538C53822E54A24E94008D2A3C256D269
:1058E000A2C2593098EFC298E5991258CE22309949
:1058F000FDC299F5991258CE22C2A3C256C2A2C2C5
:1059000059C2B675380074051258EEE51E1258EEED
:10591000E51F1258EE2212831912831912831912ED
:1059200058F9E5371258EEE5381258EE3099FD2255
:105930001209320259391208CEC0E01258F9E5377F
:105940001258EED0E01258EEE5381258EE3099FDBC
:10595000221283191258F9E5371258EE7980E712AE
:1059600058EE09DDF9E5381258EE3099FD22D216CD
:10597000754A19751A0012838FE539600B54F87057
:1059800007C227A227B392A5E53A600B54F8700727
:10599000C228A228B392A6E53B600B54F87007C258
:1059A0002CA22CB39280126E98C28EC28CC2ADC251
:1059B000ABC2ACC2AF7581D79059C3C082C08375EA
:1059C000D00032D2AFD28C127304C2ACD299125929
:1059D00016B2B5754A19D298025A00B40922F538A0
:1059E0001258D5B51E271258D5B51F211258D5B457
:1059F000461B1258D5AF381258D56F701012591671
:105A0000D2B6D2A3C256D2A2C2591258D5B40ACB2A
:105A1000F5381258D5B51EF51258D5B51FEF1258E6
:105A2000D5F537B46D03025AB6B46E03025ACFB43B
:105A30006F03025B06B47003025B53B47103025B35
:105A400067B47303025B78B47403025B7AB47503C2
:105A5000025B8EB47603025BA6B47703025BA9B443
:105A60007803025BBDB47903025BDEB47A03025BA8
:105A7000FAB46C03025C0EB46B03025C30B46A03CC
:105A8000025C6BB46903025C87B46803025CE6B431
:105A90006703025CFEB46603025D19B46503025D30
:105AA000DDB46403026521B463030264E8B46103F6
:105AB00002657C025A00AF381258D56F70F5125942
:105AC00016D2B675F01E1282E9D5F0FA0274D2121F
:105AD00058D5FD1424E0402B1258D52400FC7B003F
:105AE0001258D5FEAF381258D56F70178EF0EDF9F9
:105AF0007480F88B308C3185F03212043D1259518C
:105B0000754A19025A001258D5FD1454E070F41267
:105B100058D52400FC247140EA7B021258D5FEEDD2
:105B2000FA78801258D5F608DAF9AF381258D56FDE
:105B300070D1C2A3C256C2A2C2598EF0EDF97480D0
:105B4000F88B308C3185F03212039212591F754A4E
:105B50001980B0AF381258D56F70A81206F21259DA
:105B600016754A19025A00AF381258D56F700912CB
:105B70005936754A19025A0080891258D5FD1424E5
:105B8000E040371258D52400FC7B01025AE012583D
:105B9000D5FD1454E070231258D52400FC24254070
:105BA000197B03025B1B025B03AF381258D56F7081
:105BB00009125930754A19025A00025B0379187D9F
:105BC000071258D5F309DDFCAF381258D56F70EACB
:105BD0001267E440E51277AD12591F025A00AF3840
:105BE0001258D56F70D41277CC1283191258F9E578
:105BF000371258EE1202C8025A00AF381258D56F49
:105C00007066120CD1125916754A19025A001258B0
:105C1000D5FE1258D5FD1258D5FCAF381258D56FA5
:105C200070461206584041125916754A19025A0018
:105C30001258D5FE1258D5FDAF381258D56F7028BE
:105C40001206291283191283191258F9E5371258CE
:105C5000EEEE1258EEED1258EEEC1258EEE5381258
:105C600058EE3099FD025A00025B03AF381258D546
:105C70006F70F51283191283191258F9E53712580B
:105C8000EE1210AC025A00AF381258D56F70D9120C
:105C900008C660027401C0E012092A60027402D0D2
:105CA000F045F0700A12073D12154E120CD1E4C0F7
:105CB000E01258F9E5371258EED0E0C0E01258EE85
:105CC000E5381258EE75F0031282E9D5F0FA125851
:105CD000F9E5371258EED0E01258EEE5381258EEDA
:105CE0003099FD025A001258D5FD1454E070271265
:105CF00058D52400FC2471401D7B00025B1B125808
:105D0000D5FD1454E0700F1258D52400FC24254012
:105D1000057B01025B1B025B03AF381258D56F7025
:105D2000F51283191283191258F9E5371258EE74D7
:105D3000021258EE744E1258EE74801258EE7448E7
:105D40001258EE74311258EE74001258EE748D121F
:105D500058EE74201258EE74DA1258EE740012588D
:105D6000EE740F1258EE74A01258EE74801258EEB2
:105D700074001258EE74001258EE74201258EE742B
:105D8000001258EE74001258EE74001258EE7400AF
:105D90001258EE74001258EE74001258EE7400128D
:105DA00058EE74001258EE74001258EE7400125837
:105DB000EE74001258EE74001258EE74001258EE91
:105DC00074001258EE74001258EE74001258EEE58A
:105DD000381258EE3099FD025A00025B031258D572
:105DE000F5831258D5F5822460E58334F040EB1238
:105DF00060691258D5FD1454E070DF780075F0200A
:105E000074FFF208D5F0FB78001258D5F208DDF9DE
:105E1000AF381258D56F70C212591675F00512823C
:105E2000E9D5F0FA12591F751A013008AD12609FBA
:105E3000126085126077121A4E789879007A0A7586
:105E4000F00FE3540FF652F00809DAF643F0F0E5EC
:105E5000F00478A179847A05121929600B125EFE8C
:105E60005006751A04025DDA126085126077121A04
:105E70004E78A4790A7A0675F00FE3540FF652F0C3
:105E80000809DAF643F0F0E5F00478A979877A0397
:105E9000121929600B125F9C5006751A06025DDA12
:105EA0001260851260E8751A65025A00C0E0782811
:105EB000E583F208E582F2D0E022C0E0782AE583AB
:105EC000F208E582F2D0E022C0E07828E2F583080B
:105ED000E2F582D0E022C0E0782AE2F58308E2F51C
:105EE00082D0E022E5822400F582E583341BF5832D
:105EF00022E5822400F582E583343BF5832212609B
:105F000077AB83AC82901B00C0837900753003852A
:105F100083317532009000551203471204B8120302
:105F2000471205169000557A80E0A3F5F0E0A36CC7
:105F30007005E5F06B6017DAF0D0830583740024F8
:105F4000C0E58334C550C1740512604BD322D083A1
:105F5000EA2AF5F0E4C395F0F582125EAC78987900
:105F6000007A0A75F00FE3540FF652F00809DAF6DA
:105F700043F0F0E5F004600C121B3B700A7406124B
:105F8000604BD322121B3BE5822582F582E58335E7
:105F900083F583125EE4125EBA0262F0126077ABA0
:105FA00083AC82903B00C0837900753003858331D8
:105FB0007532009000551203471204B812034712BD
:105FC00005169000557A80E0A3F5F0E0A36C70050B
:105FD000E5F06B6017DAF0D0830583740024C0E528
:105FE0008334A550C1740512604BD322D083EA2AB2
:105FF000F5F0E4C395F0F582125EAC78A4790A7AE4
:106000000675F00FE3540FF652F00809DAF643F084
:10601000F0E5F004601D121C21701BAB83AC8212F2
:106020006077EBB58306ECB58202C322740412607C
:106030004BD322121C21E5822582F582E58335832C
:10604000F583125EF1125EBA0262F0F51A22C08286
:10605000C083E5831267E3D083D082C082C083E52A
:10606000821267E3D083D08222C0E0782CE583F2ED
:1060700008E582F2D0E022C0E0782CE2F58308E265
:10608000F582D0E02274001258EE74001258EE74BB
:10609000001258EE74001258EE74001258EE227579
:1060A000831B75821B75F040C0F0C082C0837530C1
:1060B000018583317532001203471204B8D083D0B2
:1060C00082C082C08375300385823175320012032D
:1060D0004712057ED083D08205830582D0F0D5F0AB
:1060E000C77533FF7534FF227401F97418F87530E1
:1060F0000075310075320012043D7401F97419F80D
:106100007530017531D97532FF12043DAC1812603B
:1061100077E5822420F582E583347DF583C082C053
:10612000837401F9743CF8753000858331858232BF
:1061300012043DD083D0827401F97410F8753000D8
:106140008583318582321203617810E2F5F0E5181B
:10615000253CC395F0F518126077124CFB78537903
:1061600080E2F72519F5190809E2F72519F51978DC
:10617000167953E2F3FA0809E2F32AFAC3E5199A09
:10618000F519126077124D25126077E58275F008D7
:10619000A42420F582500205F0A8F0E58375F008EC
:1061A000A4282400F5837408F97480F875300085FC
:1061B000833185823212043D7880E5187A082608FA
:1061C000DAFCF518789879007A0A75F00FE3540F25
:1061D000F652F00809DAF643F0F0E5F0041267270A
:1061E00078A4790A7A0675F00FE3540FF652F00896
:1061F00009DAF643F0F0E5F00412672F7408F97439
:1062000080F8753000858331858232120392788060
:10621000E5187A08C39608DAFBF518126077C3E52B
:106220008233F582E58333F583C3E58233F582E576
:106230008333F583E5822400F582E583245BF583CF
:10624000C082C0837404F97480F87530018583318D
:1062500085823212043DD083D0827404F97412F81E
:10626000753001858331858232120361788079121D
:10627000E5197A0426F5F0E3C5F0C395F00809DACC
:10628000F3F5197401F97418F8753000753100755B
:1062900032001203927401F97419F87530017531E6
:1062A000D97532FF12039275831B75821B75F040FE
:1062B000C0F0C082C083753003858331753200120F
:1062C00003471204B8D083D082C082C083753001E6
:1062D00085823175320012034712057ED083D08249
:1062E00005830582D0F0D5F0C77533FF7534FF22E2
:1062F000125ED6E5828583F0125EC8C39582C0E047
:10630000E5F09583D0F045F07002C322500302649B
:106310000B125ED6C0E0C3E58224FEF582E583342D
:10632000FFF583D0E0125EBAE5828583F0125EC885
:10633000B58207E5F0B58302C322125EC8AF8312AF
:106340005ED6EFB58310AE8290002C7880E0F6A385
:1063500008E0F602636E7EFE8F8305837402F97493
:1063600080F875300385833175320012043D790061
:106370007530038F317532009000551203471204B7
:10638000B81203471205168F83758200125EC87D0E
:1063900000E5836F7002AD82ED2455F582758300B0
:1063A00050020583C3EE9D20E05A03FCC082C083E7
:1063B000A3A3E0FAA3E0FBD083D082EAF0A3EBF042
:1063C000A3DCE9EE2455F58275830050020583783D
:1063D00080E6F0A308E6F079007530038F3175325E
:1063E0000090005512034712056A12034712057EFA
:1063F000853033853134125ED6EFB583030264DF16
:106400000F02633F740812604BD322125EC8AF8341
:10641000125ED6EFB58310AE8290002C7880E0F645
:10642000A308E0F602643F7E008F8315837402F9AF
:106430007480F87530038583317532FE12043D791E
:10644000007530038F3175320090005512034712EA
:1064500004B8120347120516125EC87DFEE5836F6D
:106460007002AD82ED2455F58275830050020583DC
:10647000C3ED9E20E06B03FCC0E0C3E58224FEF583
:1064800082E58334FFF583D0E0C082C083E0FAA3C5
:10649000E0FBA3EAF0A3EBF0D083D082DCDAEE24B9
:1064A00055F582758300500205837880E6F0A308D5
:1064B000E6F079007530038F317532009000551287
:1064C000034712056A12034712057E853033853172
:1064D00034125ED6EFB583030264DF1F026410C37B
:1064E00022740912604BD3221258D5F5831258D565
:1064F000F5821258D570271258D57022AF3812582D
:10650000D56F701AC01EC01F85831E85821F12188A
:10651000F0126665D01FD01E125916025A00025B97
:10652000031258D5F5831258D5F582AF381258D5D5
:106530006F70EBC01EC01F85831E85821F1218F06E
:106540007401F97480F875300075310075320012ED
:10655000043D7880E6C3951EC3951FD01FD01E252D
:106560001E251FF67401F97480F87530007531002E
:10657000753200120392125916025A001258D5F5BC
:1065800083AF381258D56F70951283191283191280
:1065900083191258F9E5371258EE74001258EEE5D7
:1065A0001A1258EE74001258EE74001258EE74006D
:1065B0001258EE74001258EEE5381258EE3099FD7C
:1065C000025A009065CBC082C083327581D775D0E6
:1065D000000274D2C082C083E5822420F582E58364
:1065E000347DF5837401F9743CF87530008583318E
:1065F000858232120392D083D082C082C083E5822A
:1066000075F008A42420F582500205F0A8F0E58377
:1066100075F008A4282400F5837404F97480F875D3
:106620003000858331858232120392A3A3A3A37421
:1066300004F97484F8753000858331858232120341
:1066400092D083D082E5824583600EE5822418E5EE
:106650008334FC74FFF5F0500BC082C083124D25CB
:10666000D083D082221208CEC0E07401F97480F881
:1066700075300075310075320012043D7880E6D027
:10668000F0C395F0F67401F97480F8753000753137
:106690000075320012039222753C007854E4F278BF
:1066A0008075F00876FF08D5F0FA22751E30751F48
:1066B00030C263C26475F005C0F0D2A3C256C2A254
:1066C000D259D2A1C258D2A4C25712669812215FE1
:1066D000D0F0205009205106D5F0DD026722126764
:1066E00047403F1200D77885E6B4FF05C32275F016
:1066F00005C0F012215FD0F0205106D5F0F30267FB
:1067000022E53DB4021C78A4E624F6401508E624F0
:10671000F6400F78A4E62430F51E08E62430F51F75
:10672000C3221200ABD322789879807A058006784C
:10673000A479857A03E608540FC4F5F0E608540FEF
:1067400045F0F709DAEF2220503130513AE53D604B
:106750000624FD24FC403012672F1200E475F0057A
:10676000C0F012215BD0F0205011204406D5F0F08B
:1067700002678712115DB40B0E8003126727753C08
:10678000007854E4F2C322D32212679975F06412A0
:1067900082E9D5F0FA12007C2275F03C12011E123B
:1067A0006E9375F03C12011E126E9875F014120172
:1067B0001E126E9375F03C12011E126E9875F01445
:1067C00012011E126E9375F01412011E126E98754E
:1067D000F01412011E126E9375F01412011E126E47
:1067E00098222222781DE254C07078E275F00A8463
:1067F000C445F07882F6781CE254C07066E275F009
:106800000A84C445F07883F6781BE254E07054E2C1
:1068100075F00A84C445F07884F6781AE26044542E
:10682000E07040E275F00A84C445F0C0E07818E2F8
:10683000030354C0D0F045F07885F67819E2602360
:1068400054F0701FE275F00A84C445F0C0E0781E71
:10685000E254F8700EE2C42354E0D0F045F078869C
:10686000F6C322D32290000075F019C0F07402F92B
:106870007480F875300185833185823212043D7849
:1068800081B6FF02800E18E552300805B4FF02E51C
:1068900064666011E5822410F58250020583D0F011
:1068A000D5F0C8C322D0F0A3D32230084DE582240E
:1068B000FFF582E58334FFF58375F019E5822480C6
:1068C000E58334FE5005900000800AE5822410F52F
:1068D0008250020583C0F07402F97480F8753001AB
:1068E00085833185823212043D7881B6FF028005AE
:1068F00018E6B55207D0F0D5F0C2C322D0F0A3D32A
:106900002222300F0CC20F1267E440051277AD80CF
:10691000031277CC7885E6C45403E6540F7886E6F4
:10692000C45401E6540F7884E6C4540FE6540F783B
:1069300083E6C4540FE6540F30080A126865500508
:1069400012690180031269B122C2AC127304C2AC95
:10695000128319128319D299C2B674FF1258EE75B8
:10696000380074421258EE74621258EE74151258C0
:10697000EE742A1258EE741B1258EE74001258EE80
:1069800074001258EE74001258EE74001258EE1291
:1069900002D575F010C0F074001258EED0F0D5F0AA
:1069A000F4E5381258EE3099FDC24FD2B612730496
:1069B0002222201401227475787912012F501A2096
:1069C0006819D268126F677518C075190B741A545C
:1069D0003F4400F51A1209C422C2681277CC203352
:1069E00004203433227884E6543FF5F0796FE36570
:1069F000F0702109E3788366701A203516D23512BB
:106A00006F677518C075190B741A543F4400F51A56
:106A10001209C42230342F7884E6543FF5F079719E
:106A2000E365F0702109E3788366701A203516D289
:106A300035126F677518C075190B741A543F4400EE
:106A4000F51A1209C422C23522C2AC120A02600C25
:106A5000F5188819120D44120A1A80EFD2AC227E62
:106A6000007F8490000075F000E49325F0F5F0A31A
:106A7000C3E5829EE5839F40F0E5F070022200E5C9
:106A8000F0C0E0E5831267E3E5821267E3D0E0122D
:106A900067E3C2ADC2ACD216C2A012009420B7F810
:106AA00075F0C81282E9D5F0FA30B7FD75F0C8125A
:106AB00082E9D5F0FA1273042275F032128301B222
:106AC000B5128301B2B5D5F0F32275F064120591C9
:106AD00020E50430E30122C2AFB2B5128301B2B5A2
:106AE000128301D5F0E7126E93126AB9126E9812F2
:106AF0006AB9126E93126AB9126E98126AB9126A62
:106B0000B9126AB9126AB980DD2230083C74007883
:106B10008912013E40337F087E0074787879120133
:106B20002FCE13CE05E0DFF420170E7400789912F3
:106B3000013E5005EE655460108E548E527518C09B
:106B400075190485521A1209C422C2AF751810753E
:106B5000190FF51A1209C4D2AF22223008FC205CAA
:106B6000F97401788912013E40F074777879120146
:106B70002FE492E0C0E07476787912012FD0E033F0
:106B8000FE20170E7401789912013E5005EE6555EE
:106B900060C88E55EE20E10630E028026BD630E06A
:106BA00014A25E725D50B3C25EC25D126E7774F85D
:106BB000126B4A80A5D25EC25D126E7774F7126BBB
:106BC0004A8097205D0ED25DC25E126E77D25B74F2
:106BD000F6126B4A8084A226825D40F8D25DC25EC6
:106BE000126E8B74F5126B4A026B5AC082C083D04E
:106BF00083D0822222304309C2A3C256D2A4C257F4
:106C000022D2A3C256C2A4C25722200801223008B1
:106C100019C0E0C082C0837407120188D083D0827B
:106C2000D0E04003026C48026C2A20170820603331
:106C3000D260205F2ED25FD2607518C075190075C2
:106C40001A0F1209C4026C63201708306015C26065
:106C5000305F10C25FC2607518C0751900751A10D8
:106C60001209C4300819C0E0C082C083740F120139
:106C700088D083D082D0E04003026C9D026C7F20DC
:106C80001708206233D26220612ED261D262751859
:106C9000C0751900751A511209C4026CB820170882
:106CA000306215C262306110C261C2627518C0756F
:106CB0001900751A521209C422C2B675380074033D
:106CC0001258EEE51E1258EEE51F1258EE744E12E1
:106CD00058EE74081258EE74011258EE74061258E9
:106CE000EE7848E2F5F0E5F01258EE08E2F5F0E54E
:106CF000F01258EE784AE2F5F0E5F01258EE08E2AC
:106D0000F5F0E5F01258EE2442F8E2784CE2547FB8
:106D1000F5F07844E2C36001D3E5F092E7F5F0E5E1
:106D2000F01258EE75F000E5F01258EEE538125802
:106D3000EE3099FD22C2B6127CD5127C6475380003
:106D400074031258EEE51E1258EEE51F1258EE7449
:106D50004E1258EE740C1258EE74001258EE740A6B
:106D60001258EEC082C083A3A3A3E49375F064A479
:106D7000C0E0E5F01258EED0E01258EEA3A3A3A3B2
:106D8000E49375F064A4C0E0E5F01258EED0E01290
:106D900058EED083D082E4931258EEA3E4931258B5
:106DA000EEA3A3A3E4931258EEA3E4931258EEE5E6
:106DB0008D1258EEE58B1258EEE5381258EE3099E8
:106DC000FD22C2B6121304C0E075380074031258D5
:106DD000EEE51E1258EEE51F1258EE744E1258EEF4
:106DE00074041258EE74021258EE74021258EEE552
:106DF0007E1258EED0F0E5F01258EEE5381258EE5B
:106E00003099FD22C2B6121242C0E07538007403F8
:106E10001258EEE51E1258EEE51F1258EE744E128F
:106E200058EE74041258EE74021258EE740212589E
:106E3000EEE57E1258EED0F0E5F01258EEE538128D
:106E400058EE3099FD22C0F088F0C0F0C2AF7576E0
:106E5000007850E2F54CF5F008E2F54DD2AF45F080
:106E6000D0F0A8F0D0F07009B226202604126E816E
:106E700022D22675760322C2AF754CFF754DFFD224
:106E8000AF757600C209C226D2A722126E46D25B27
:106E9000D25522C26E028249D26E028249305D1200
:106EA00020260F543F4400F51A7519087518C012B2
:106EB00009C422C0E0C8C0E0E47868F208F2D0E07B
:106EC000F8D0E022C0E0C8C0E0E87869F218E4F247
:106ED000305D0820260578687401F2D0E0F8D0E033
:106EE00022C0E0C8C0E07868E2601408E2543F4481
:106EF00000F51A7519087518C01209C4126EB3D0BE
:106F0000E0F8D0E022D2B2C2B4D293C322D2B2C24D
:106F1000B4D29312830120B2ECC29312830130B237
:106F2000E4D29312830112830120B2D9C293128357
:106F30000112830130B2CED2B2C2B4D293D32212A4
:106F40000488C28474541204A2E412046212047508
:106F5000F5F06448255E33F55EE5F0255FB2E003A9
:106F6000F55FD9E9D284227583DD75F010753003A1
:106F7000858331753200C083C0F012034712086068
:106F8000D0F0D0830583D5F0E47533FF7534FF75F9
:106F9000770075780022E5822400C0E0E58334DDC7
:106FA000F8D0E0C322C082C0837401F97480F87500
:106FB000300385833185823212043D7880B6020C1D
:106FC000E57824FFF578E57734FFF577D083D08234
:106FD00022126F96C082C083F5828883126FA578D3
:106FE0008076007401F97480F875300385833185EB
:106FF0008232120392D083D08222126F96C082C056
:1070000083F5828883C082C0837401F97480F87527
:10701000300385833185823212043D7880B60209BF
:10702000D083D082D083D08222E5782401F57850B5
:10703000020577D083D082788076027401F974805B
:10704000F8753003858331858232120392D083D064
:107050008222126F96126F96C082C083F582888357
:10706000126FA5788076017401F97480F875300389
:10707000858331858232120392D083D08222126FAF
:1070800096C082C083F5828883126FA578807603CC
:107090007401F97480F8753003858331858232126A
:1070A0000392D083D08222126F96C082C083F58271
:1070B00088837401F97480F8753003858331858283
:1070C0003212043D7880E6B40102800CB4020280E2
:1070D00007B4030280027400D083D0822212048895
:1070E000C28474541204A2E4120462120475B4023D
:1070F00005755E018002D9F3D28422755E00758326
:10710000DD75F00F753003858331753200C083C0A3
:10711000F01203471204B812034779001270DDD051
:10712000F0D0830583E55E7026D5F0D875300385F1
:1071300083317532001203471204B812034779A055
:107140001270DD7533FF7534FFE55E7002D322C324
:1071500022E578457760167866E2F5F008E245F0BA
:10716000600BD37867E2957818E2957722C32212F4
:1071700070A7C2B675380074031258EEE51E125897
:10718000EEE51F1258EE74501258EE747D1258EE50
:10719000900000E536600F9003E81460099007D076
:1071A000146003900BB87E7D7F0875F000C0F0126C
:1071B00070A7B40203D38001C3D0E033F5F0A3DF9E
:1071C000EC1258EEDEE2E5381258EE3099FD22C29C
:1071D0008C758A45758C5DD28CB20020000132C05E
:1071E00000C0D0C0E0C0F075D008D25412115C12BB
:1071F00072E5051DE51D20E00C20E109301618E5BB
:107200001D541F6054201604E54B6002B2B5D0F047
:10721000D0E0D0D0D00032205905A226B392A2E50A
:107220001D30E203127F8AE51D541F702FD255C214
:107230007278AAE2D5E006D271D272743CF2C082B2
:10724000C083127E76D083D082E4B54745B54957D6
:10725000B5635FB56F60B57F64B54A65E4B54B4310
:10726000B5486CB5456DB54E71B57672E54D454C7A
:10727000601DE54D2401F54D5002054C454C700F45
:10728000C209205C0A205D07126E81D25BD25502D2
:107290007205D547B8C2097549B4757D00D247D289
:1072A0004A80AA154B80B9D549A6C245C246C247F5
:1072B000809E1563809DD56F9DC2708099157F80DB
:1072C00098D54A987546033016030265C380811528
:1072D000488090D54590D24E808C154E808BD576C7
:1072E0008BC2A78087E51DA2E330560292A33059D6
:1072F0000292A230580292A122C2B6204F02D2B608
:107300001273043275C800C2ADC2AC75CBFF75CA2A
:107310009875CDFF75CC98759853C298C299D2AC28
:10732000C2BC75C8347599062275C800C2ACC2AD1E
:1073300075980075CC2B75CDEBD2AD75C804227550
:10734000C800C2ACC2AD759800E58A242BF5CC54B8
:107350000F658C24EBF5CDD2AD75C80422C2A8C24E
:10736000AAC289C28BC2ACC2A9C2AB758F01120579
:107370009ED216126E98126E77E4F53C7854F2782D
:107380007975F010F2D5F0FCC25CC25DC25EC25FDE
:10739000C261753EFF7540FF751D04C244C245C2FF
:1073A00046C247754901754A00C24AD254757300F6
:1073B000C235C218C219D24EC24F754510E4F5410C
:1073C000F542F543F535F537121ED8751E00751FC9
:1073D00080E4F547F550F54FF558F559F53FC223D0
:1073E000C224C225C22B74377859F2785AF2785BDE
:1073F000F2785CF2D21F75460375480178AC7A05C5
:1074000076FF08DAFBC20F7818E47A07F208DAFC94
:10741000C2107552FF855254C211C208757F0375A0
:10742000631E756500C267C20DC20EC209C20AC2E0
:107430000BC263C26475610075600075F006784226
:10744000E4F208D5F0FB7948E4F309F3794AF3094B
:10745000F3784CE4F2121476754BFAB2B57533FF3B
:107460007534FFD268756E007827740AF2127CB406
:10747000C270756F0175721AC201C202C203C204E2
:10748000C205D2A075760075770075780078A9746A
:10749000FAF2E478B1F278B2F278B3F278AA743CF6
:1074A000F2C274C273C26F757D00127DE9C275D2DB
:1074B00076C277758901758A3E758C5DC2B9D2A98D
:1074C000D28CD2B6127304D2AFD293C2B4D2B2B2BB
:1074D000B522C21675510375F0031282E9D5F0FA90
:1074E000C263C26412369875510375F0031282E9C3
:1074F000D5F0FAC263C264123537C2AF0200002071
:10750000051320040820020D200102C32212148A50
:107510001278BFD3221279C8D32275F000C0F012BE
:107520002361D0F0500343F008E5F02230731420BB
:10753000431D78B3E2307106C271600214F224FA7E
:10754000500422307409E57C540170031200E422D7
:10755000C274C273E478B3F222C2AF754BFAB2B50B
:10756000128301B2B5128301B2B5D2A07581D7756D
:10757000D00012735D126BEB126A5F126F67121DFF
:107580004B754BFA120C421274FF755103123812EC
:107590001238281200F1751880751904751A8012B6
:1075A00009C4D21730080F120A92126B0A126B5BD1
:1075B0001269B2126C0AD2B7D2AFC216C21700005B
:1075C0000020B70912830120B703021D653008327D
:1075D000120A9212752CE57A5420601178A9E2D52E
:1075E000E00A1277CC12694978A974FAF2E57D6055
:1075F00002157D30080C126B0A126B5B1269B21215
:107600006C0AE5656003D5650B127DE212390C1238
:107610006902800CD2A3C256C2A1D258D2A4C257CA
:10762000E5637003126A49C259D2A1C258126BF5C0
:10763000C263C264D25B785FE2600D24FD400975CD
:1076400075021239FB1274FF7860E2600D24FD4070
:10765000097575031239FB1274FFE5795440600611
:1076600020A80312338212215F20510820500520E8
:107670005202801A302F09304606126BEB027686D2
:1076800012451C1274FF7827E215E0F27008782783
:107690007414F20275B60275ED0074A212772EE82A
:1076A000127769E91277691277A02274A212772EF5
:1076B000E8127769E712776909D582F81277A02274
:1076C00074A212772EE812776974A312772E1277BC
:1076D00089F709D582041277A022C296D2970000BA
:1076E00000C29780E974A212772EE81277691276A9
:1076F000F22274A312772E127789F91277A02274DE
:10770000A27A08C296000000C297335005D29602B2
:107710007714C296D297000000C297DAEDD2960095
:10772000D297000000309604C297C322D3227A0871
:10773000D296D29700000000000000000000000078
:1077400000000000C296000000C297335005D29698
:10775000027755C296D297000000C297DAEDD29612
:1077600000D297000000C297227A08335005D296C3
:10777000027775C296D297000000C297DAEDD296D2
:1077800000D297000000C297227A08D296C29700D2
:10779000000000D297C3309601B333DAF0C29722CB
:1077A000C296000000D297000000D2962278807620
:1077B000000876007884E6543FF678007980C0822D
:1077C0007582071276ABD0821282E9227802798222
:1077D000C0827582051276C0D082227886E603C404
:1077E000540775F018A4C0E07884E6C4540375F01B
:1077F0000AA4F5F0E6540F25F0D0F025F075F03C22
:10780000A4C0F0C0E07883E6C4540775F00AA4F57C
:10781000F0E6540F25F0D0F025F0F5F0D0E034007C
:10782000C5F022207556206921C0D0C0E0E8C0E034
:10783000C0F0E54E7003857270754E08D26C1279F7
:107840003BD0F0D0E0F8D0E0D0D0C2893220692916
:10785000C0D0C0E0E8C0E0C0F0E54E700375700035
:10786000754E08A2B2B3926C127A20308502D20310
:10787000D0F0D0E0F8D0E0D0D0C28B32C2A8C2891C
:10788000322075C9206926C0D0C0E0E8C0E0C0F051
:10789000E54E7003857270754E08C26C12793B30EC
:1078A0008502D203D0F0D0E0F8D0E0D0D0C28B3245
:1078B000C2A8C2AAC293C2B4C0E01282E9D0E0C298
:1078C00075C293C2B4C289C28BD2B2D2B3C2697537
:1078D0004E00857270C203C2B8D288D2A8C2BAD292
:1078E0008AD2AA22C275C2A8C2AAC289C28B22E5C4
:1078F00072141475F00884F5F0C0F0782EE230E0D0
:1079000002B26A30E102B26A30E202B26A30E302E5
:10791000B26A08D5F0E7D0F0E230E002B26B30E1B5
:1079200002B26B30E202B26B30E302B26B08D5F008
:10793000E7206A05306B02C322D322E570B57207D7
:10794000A26C926A027985B40107A26C926B0279EB
:1079500085C3E572149570403275F00484242EF8C6
:10796000E205F0D5F006A26C92E38016D5F006A2EF
:107970006C92E2800DD5F006A26C92E18004A26CBC
:1079800092E0540FF2D57002D26922857270D269EA
:10799000227548321278B0305405C25412027AE58A
:1079A0004860113069F1E570700A1278E41278EFDE
:1079B0004002C3221278E4D322C2A8C2AAC293C250
:1079C000B4C0E01282E9D0E0D275C293C2B4C289D9
:1079D000C28BD2B2D2B3C269754E00757000C203B9
:1079E000C2BAD28AD2AA227548321279B930540565
:1079F000C25412027AE548600C3069F1E5707005F6
:107A00001278E4C3221278E4D322C330E001B33009
:107A1000E101B330E201B330E301B330E401B3225A
:107A2000E57075F00584C0E024ECD0E04055242ECC
:107A3000F8E2A26C92E503F2E570700BE2541FB419
:107A40000B40757005803B0570E5F0B40434E2121C
:107A50007A0A502F540FF218E2540FB40F24D3E8CF
:107A6000942E782EF20404C082F58275F00B08E2A1
:107A700065F0F5F0D582F7D082540F7006D26975A3
:107A80007000221279C822010000000000000000EE
:107A9000000A0000000000000000000406000000D2
:107AA0000000000000080E030000000000000000BD
:107AB000010702000000000000000A0608010000A3
:107AC000000000000402040F00000000000008068F
:107AD000090809000000000000010E050F05000064
:107AE0000000000A0C0A090B0300000000040E0B42
:107AF00000040502000000080E0607080407010044
:107B0000000001050A040D080E75F00A7998770047
:107B100009D5F0FA782EE2FA60400824F25007EA1C
:107B200024F328F87A0DE2540FF26029EA1475F074
:107B30000AA42487F5827400347AF58379A17E0043
:107B40007B0AE493F5F0E2A42E2775F01084FEA7DB
:107B5000F0A319DBED08DACEC322D322094300A03B
:107B60000954009F0966009E0977009D0989009CC1
:107B7000099B009B09AD009A09BF009909D20098A2
:107B800009E4009709F700960A0A00950A1D009477
:107B90000A3000930A4300920A5700910A6B009042
:107BA0000A7F008F0A93008E0AA7008D0ABB008C03
:107BB0000AD1008B0AE7008A0AFE00890B140088AC
:107BC0000B2B00870B4300860B5C00850B75008434
:107BD0000B8E00830BA700820BC100810BDB0080A2
:107BE0000BF6007F0C10007E0C2B007D0C47007CF8
:107BF0000C64007B0C81007A0C9E00790CBB007831
:107C00000CDB00770CFB00760D1B00750D3B007440
:107C10000D5B00730D7D00720D9F00710DC2007031
:107C20000DE4006F0E07006E0E2C006D0E51006CFF
:107C30000E76006B0E9B006A0EC100690EE90068AB
:107C40000F1100670F3900660F6100650F8900642E
:107C50000FB300630FDE0062100900611034006092
:107C6000105F005F7F42907B5CE493A3F5F0E493A8
:107C7000A3C3958BE5F0958D5015A3A3DFEBE582AB
:107C800024FFF582E58334FFF583E49314800BA38E
:107C9000E493BF4205907B5C8010C0E0E58224F94C
:107CA000F582E58334FFF583D0E02290006AE0A2FC
:107CB0008733F02290006B7400F090006A7455F0E6
:107CC00090006C74FFF090006E7405F090006D747D
:107CD00012F0D28122D286A2A4C0D0D2A475F00024
:107CE000D5F0FDD5F0FDC28E53890F438910758BF9
:107CF00000758D00C28FC2AFC2A4D28E2086033021
:107D00008FFAC28E308F06758BFF758DFFD2AFD084
:107D1000D092A422F024FE4005308102C28122903C
:107D2000006EE0D5E0EE7442F0127CD5D281E58B96
:107D30002499E58D34F24014E58B24E1E58D34F38C
:107D4000400EE58B24E0E58D34FC40087415800678
:107D5000741180027412FE90006DE06E6013EEF0FC
:107D6000E5795404700B7518C07519008E1A120944
:107D7000C422127CAB603904603690006CE020E0D5
:107D800010D2E0F090006BE070047405F022E4F093
:107D90002290006BE0602C14F07028E5795402709A
:107DA000227518C0751900751A141209C4027DC312
:107DB00090006CE030E00DC2E0F090006BE070CE1F
:107DC000743CF02290006BE060F914F070F5E579F6
:107DD000540270EF7518C0751900751A131209C492
:107DE00080E1127D1F127D72229002EB75F008E493
:107DF000F0A3D5F0FB9002F375F00874FFF0A3D563
:107E0000F0FB22C0E0127E56D0E0B3502CC0E0243C
:107E1000F8D0E04022C082C083F5F024F3F582E47C
:107E20003402F583E0C5F024EBF582E43402F583F7
:107E3000E5F0F0D083D082D322C0E024F8D0E04037
:107E400013C082C08324EBF582E43402F583E4F0AE
:107E5000D083D082C322C0E024F8D0E04016C08294
:107E6000C08324EBF582E43402F583E0D083D08232
:107E70006002D322C3229002EB75F008E06003B4E5
:107E8000FF05A3D5F0F62220E70414F080F4307249
:107E9000F114F0B480ECE4F080E8B4400774001210
:107EA0007E56803DB441077401127E568033B44241
:107EB000077402127E568029B443077403127E565B
:107EC000801FB444077404127E568015C0E024E479
:107ED000D0E04013232452C0E07400347FC0E0227D
:107EE000C3740122D380FAE4C322A243B380F2D246
:107EF00055A26F80EC80F0A20980E6A20B80E2A27E
:107F00007780DE80DF80E0A20A80D63070D280D415
:107F1000E577457860CA80CC12715180C4A25E7248
:107F20005DB380BDA25D822680B7A25DB02680B120
:107F3000A25E80ADC330730920430678B3E27001BE
:107F4000D3809EA26EB38099C3E57F6001D38091F8
:107F50008095809680998097809580938091808F7E
:107F6000808D809180918093809580978097809775
:107F70008099809C80A280A580AA80AE80B280B4C7
:107F800080C180C480CA80C880C612809F30081912
:107F9000C0E0C082C0837404120188D083D082D034
:107FA000E04003027FC8027FA9E539B40D0A302101
:107FB000028035D221D3801EB4160678D2E6C38063
:107FC00015127E9A6022800EE539B40D0620210339
:107FD000027FE8C221C34009C227A227B392A5802D
:107FE00007D227A227B392A5300819C0E0C082C0EB
:107FF000837405120188D083D082D0E040030280D0
:1080000023028004E53AB40D0A3022028035D222E0
:10801000D3801EB4160678D3E6C38015127E9A600C
:1080200022800EE53AB40D06202203028043C222CC
:10803000C34009C228A228B392A68007D228A2284A
:10804000B392A6300819C0E0C082C083740B12013D
:1080500088D083D082D0E0400302807E02805FE53A
:108060003BB40D0A302A028035D22AD3801EB416C2
:108070000678D4E6C38015127E9A6022800EE53B16
:10808000B40D06202A0302809EC22AC34009C22CD6
:10809000A22CB392808007D22CA22CB3928022B261
:1080A0000C300C60E57A5410600330431BE57B54C0
:1080B000047003204538E57B54017003204611E528
:1080C0007B54027003204717C26F75500002810471
:1080D000E550B401028024755001754F40801CE5C5
:1080E00050B402028015755002754FA0800DE55006
:1080F000B403028006755003754FF0E54F23F54F2A
:10810000A2E0926F22C227A227B392A522D227A271
:1081100027B392A522B227A227B392A522F5F00396
:1081200003543FB40258E53964086005E539B40DDD
:108130004AE5F089F0C0F0300819C0E0C082C08381
:108140007404120188D083D082D0E040030281629F
:10815000028153D0F0A9F05403B4020D128105023C
:108160008247D0F0A9F0028247B4010612810D02C5
:108170008247B40306128115028247028245B40386
:1081800062E53A64086005E53AB40DEFE5F089F080
:10819000C0F0300819C0E0C082C0837405120188A5
:1081A000D083D082D0E040030281C10281AED0F002
:1081B000A9F05403B40211C228A228B392A60282E5
:1081C00047D0F0A9F0028247B4010AD228A228B30E
:1081D00092A6028247B40309B228A228B392A680CD
:1081E000668062B4045FE53B64086005E53BB40D5E
:1081F00054E5F089F0C0F0300819C0E0C082C083B7
:10820000740B120188D083D082D0E0400302822513
:10821000028213D0F0A9F05403B4020FC22CA22C96
:10822000B392808022D0F0A9F0801CB40109D22C36
:10823000A22CB392808010B40309B22CA22CB3926A
:108240008080048000D322C322C0E07417306E21E6
:10825000B53907C227A227B392A5B53A07C228A20B
:1082600028B392A6B53B07C22CA22CB39280D0E0D3
:1082700022B53907D227A227B392A5B53A07D2284B
:10828000A228B392A6B53B07D22CA22CB39280D0E1
:10829000E022B4010775190F751AE122B4020775BF
:1082A000190F751AE222B4030775190F751AE32224
:1082B000B4040775190F751AE422B4110775190F64
:1082C000751AD122B4120775190F751AD222B41378
:1082D0000775190F751AD322B4140775190F751A7B
:1082E000D42275190F751AD422C28E53890F43896F
:1082F00010758BD6758D97C28FD28E308FFDC28E42
:1083000022C28E53890F438910758BEB758DCBC2BA
:108310008FD28E308FFDC28E22C28E53890F438939
:1083200010E58AC4242BF58B758DEBC28FD28E306D
:108330008FFDC28E22543F4400F51A75190A751834
:10834000C00209C4543F4480F51A75190A7518C053
:108350000209C4543F4400F51A75190C7518C0027F
:1083600009C4543F4440F51A75190C7518C0020928
:10837000C4543F4480F51A75190C7518C00209C41D
:10838000543F44C0F51A75190C7518C00209C4741D
:1083900001127E397404127E3922000000000000B0
:1083A00000000000000000000000000000000000CD
:1083B00000000000000000000000000000000000BD
:1083C000000000000000000000000000000050520B
:1083D000343032207665722E3132382E312E3020F4
:1083E0004864773A482032302D30362D30352032EF
:1083F000333A323220200043524300000000006E26
:00000001FF
:0300000306028072
